:020000040800F2
:10000000D894002005020008F53C0008F1360008ED
:10001000193C0008A90A00082D4F00080000000044
:100020000000000000000000000000004501000882
:10003000EB0A000800000000A10100085546000876
:100040001F0200081F0200081F0200081F0200080C
:100050001F0200081F0200081F0200081F020008FC
:100060001F0200081F0200081F020008AD0A000856
:10007000BD0A00081F0200081F0200081F02000836
:100080001F0200081F0200081F0200081F020008CC
:100090001F02000800000000000000001F0200080E
:1000A0001F020008894600081F0200081F020008FE
:1000B0001F0200081F0200081F0200081F0200089C
:1000C0001F0200081F0200081F0200081F0200088C
:1000D000ED3E00081F0200081F0200081F02000872
:1000E0001F0200081F020008000000001F02000895
:1000F0001F0200081F0200081F0200081F0200085C
:100100001F0200081F0200081F0200081F0200084B
:100110001F0200081F020008994600081F0200087D
:100120001F0200081F0200081F0200081F0200082B
:10013000DFF80CD000F0D2F9004800471D5100084C
:10014000D89400202C4B19680868B0E8F04F80F371
:100150000988BFF36F8F4FF0000080F3118870475C
:100160000000000008480068006880F308884FF02D
:10017000000080F3148862B661B6BFF34F8FBFF3FF
:100180006F8F00DF00BF00BF08ED00E0DFF80C005C
:10019000016841F470010160704700BF88ED00E024
:1001A000EFF30980BFF36F8F134B1A681EF0100F27
:1001B00008BF20ED108A20E9F04F106009B44FF01D
:1001C000500080F31188BFF34F8FBFF36F8F06F09D
:1001D000DBF84FF0000080F3118809BC196808684B
:1001E000B0E8F04F1EF0100F08BFB0EC108A80F39B
:1001F0000988BFF36F8F70474C640020EFF30580D0
:10020000704700000648804706480047FEE7FEE7C3
:10021000FEE7FEE7FEE7FEE7FEE7FEE7FEE7FEE7B6
:10022000654600083101000840EA01039B0703D03E
:1002300009E008C9121F08C0042AFAD203E011F825
:10024000013B00F8013B521EF9D27047D2B201E0E7
:1002500000F8012B491EFBD270470022F6E710B5CB
:1002600013460A4604461946FFF7F0FF204610BD24
:100270002DE9FE4F81EA030404F0004421F000411F
:1002800000944FF0000B23F0004350EA01045ED0CD
:1002900052EA03045BD0C3F30A54C1F30A552C4459
:1002A000A4F2F3340194A0FB0254C1F3130141F40E
:1002B0008011C3F3130343F4801301FB024400FBDA
:1002C000034E840A970A44EA815447EA8357A4FB01
:1002D000076802958D0A05FB07854FEA932C04FBFE
:1002E0000C542705029D4FEA065847EA1637B5EB2E
:1002F00008056EEB070C870E920E47EA811742EA5B
:100300008312A7FB0201B6EB0B0164EB00042B0D7B
:1003100043EA0C335E1844EB1C50DA465146E7FBC7
:100320000201C5F313044FEA0B3343EA14534FEAB7
:100330000432019C43EA0603A4F10C040294009CDD
:10034000CDE900B400F07BF803B0BDE8F08F0020E9
:100350000146F9E700F0004230F000400AD0C10D3C
:1003600001F56071C0F3160042EA0151C20840076E
:100370001143704700200146704701F0004330B43C
:1003800021F0004150EA010206D00A0DA2F5607288
:10039000C1F31301002A02DC30BC00207047440F77
:1003A00044EAC104C100E01830BC00EBC250AFF316
:1003B00000800029A8BF7047401C490008BF20F0FA
:1003C0000100704710B4B0FA80FC00FA0CF050EA5B
:1003D000010404BF10BC704749B1CCF1200421FADC
:1003E00004F411FA0CF118BF012121430843A3EBD7
:1003F0000C01CB1D4FEA00614FEA102042BF0020E4
:1004000010BC704700EBC35010440029A4BF10BCBF
:100410007047401C490008BF20F0010010BC704725
:1004200010B5141E73F1000408DA401C41F10001FC
:1004300092185B411A4301D120F0010010BD2DE953
:10044000F04D92469B4611B1B1FA81F202E0B0FA4A
:1004500080F22032904600F053F804460F4640EAFE
:100460000A0041EA0B0153465A46084313D011468D
:1004700053EA010019D0C8F14002504600F04FF88D
:1004800005460E4650465946424600F039F80843A4
:1004900005D0012004E020463946BDE8F08D00205B
:1004A000054346EAE0762C4337430A986305E40A9D
:1004B000A0EB08000022FD0A44EA47540A3002D5A6
:1004C00000200146E9E7010510196941DDE9084509
:1004D00000196941BDE8F04DA2E70000064C074D48
:1004E00006E0E06840F0010394E807009847103404
:1004F000AC42F6D3FFF720FE74750008947500082F
:10050000202A04DB203A00FA02F1002070479140D3
:10051000C2F1200320FA03F3194390407047202AC8
:1005200004DB203A21FA02F00021704721FA02F39D
:10053000D040C2F12002914008431946704770B57F
:100540008D1810F8014B14F0030201D110F8012BA3
:10055000231106D110F8013B03E010F8016B01F8FC
:10056000016B521EF9D1ABB110F8012B04F00C0451
:100570008A1A0C2C03D0A2EB84129B1C08E010F802
:10058000014BA2EB0422F8E712F8014B01F8014BF2
:100590005B1EF9D5A942D4D3002070BD70B50446C6
:1005A00000252068806800F00100F0B120688068B4
:1005B00020F001002168886001F056FC05460EE03D
:1005C00001F052FC401B022809D9E06A40F01000FB
:1005D000E062206B40F001002063012070BD2068C4
:1005E000806800F001000028EAD10020F6E7000052
:1005F00038B504460025002000902068806800F08F
:10060000010000283AD12068806840F0010021688C
:1006100088606FF010002168086040102168086051
:10062000174800681749B0FBF1F000EB800080002C
:10063000009002E00098401E009000980028F9D138
:1006400001F012FC054613E001F00EFC401B0228ED
:100650000ED9E06A40F01000E062206B40F001002B
:10066000206300BF002084F8280000BF012038BDAF
:100670002068806800F001000028E5D00020F6E73F
:100680000000002040420F0000B589B00020069015
:1006900007900890142101A8FFF7DFFD00BF2B4849
:1006A000806940F40070294988610846806900F437
:1006B0000070009000BF00BF02200190244803900A
:1006C00001A801F055FE2348234908600020486036
:1006D0000021214881604FF48071C16000210174C4
:1006E00001214161002101760121C1614FF46021A6
:1006F000016200F0A7FD08B100F030F8012006907B
:1007000007900420089006A9134800F0E7FC08B100
:1007100000F024F80220069007900420089006A913
:100720000D4800F0DBFC08B100F018F80920069035
:10073000032007900420089006A9074800F0CEFC8B
:1007400008B100F00BF809B000BD00000010024035
:1007500000C00010002401400465002000BFFEE737
:1007600010B501F06FFC10BD70B5C2B048227349DE
:1007700030A8FFF759FD48211EA8FFF76EFD28227B
:100780006E49483114A8FFF74FFD28226B4970319C
:100790000AA8FFF749FD28216846FFF75EFD0024FF
:1007A0000026002566486749886067488860674872
:1007B000C8606748C860674867490860674861491A
:1007C000C1F88C0200BF16E0032600BF30A850F825
:1007D00024000568E84380B2B0EB154F03D11EA892
:1007E00040F8245002E0701E061EEFD100BF0EB983
:1007F000FFF7B6FF641C122CE6D31E98C0F30B0063
:100800001F99C1F30B0140EA014000902098C0B24B
:100810000190219800F00F00229901F01F0140EA99
:10082000014002902398C0F30A002499C1F30C01FF
:1008300040EA014003902598C0F30A002699C1F3CD
:100840000A0140EA01400490279800F03F002899EF
:1008500001F03F0140EA01400590299800F03F0077
:100860000690DDE92A0161F31F400790DDE92C01C4
:1008700061F31F4008902E98C0F30B002F99C1F32D
:100880000B0140EA0140099000241BE014A850F835
:10089000240005685DF824100AA850F824002840B8
:1008A00081420ED014A850F8240000680AA951F81B
:1008B000241088435DF82410084314A951F824102B
:1008C0000860641C0A2CE1D323488C38006840F08F
:1008D00001001C49C1F8000200BF00BF00BF00BFFB
:1008E00000BF00BF00BF00BF00BF00BF1548D0F869
:1008F000000220F001001349C1F8000200240EE0BC
:1009000014A850F8240005685DF824100AA850F8CF
:1009100024002840814201D0FFF722FF641C0A2CEA
:10092000EED30848406940F08040064948610846D7
:10093000406940F00040486142B070BDCC6E000894
:100940002301674500200240AB89EFCD3B2A1908FF
:100950007F6E5D4C51407F5D8C2202406327CE4606
:1009600000B591B02C2106A8FFF777FC142101A84F
:10097000FFF773FC1F200690002007900C900120C9
:100980000B90002009900D9002200E9000210F91F5
:100990004FF42011109106A801F028FF08B1FFF7CD
:1009A000DDFE0F20019002200290002003900490B1
:1009B0004FF480600590042101A801F097FD08B173
:1009C000FFF7CCFE11B000BD00B587B0142102A81E
:1009D000FFF743FC00BF002001902F48C06940F49E
:1009E00000302D49C8610846C06900F4003001900C
:1009F00000BF00BF29482A4908604FF4E130486031
:100A0000002127488160C160016181610C21416141
:100A10000021C161002022490862084602F0B6FDAB
:100A200000BF1D48406B40F020001B49486308464A
:100A3000406B00F02000019000BF00BF00BF0846DF
:100A4000406B40F0200048630846406B00F02000F7
:100A5000019000BF00BF20200290022003900120DF
:100A60000490032005900220069002A90D4801F091
:100A700009F9402002900220069002A9094801F0DD
:100A800001F901220021262001F08AFA262001F036
:100A900073FA07B000BD000000100240004400409F
:100AA0006C670020000C004800BFFEE710B502494B
:100AB000C86C00F087FE10BDAC650020704730B5F3
:100AC00090F840500124AC40C56B6C6004686360D2
:100AD0004468102C04D10468A2600468E16003E05B
:100AE0000468A1600468E26030BD704700B587B05B
:100AF000142102A8FFF7B1FB00BF6948406B40F02A
:100B00000800674948630846406B00F00800019000
:100B100000BF00BF00BF0846406B40F004004863C0
:100B20000846406B00F00400019000BF00BF00BF0A
:100B30000846806940F0010088610846806900F03D
:100B40000100019000BF00BF00BF0846C06940F42B
:100B50008040C8610846C06900F48040019000BF31
:100B600000BF00BF0846406940F0010048610846E8
:100B7000406900F00100019000BF00BF4FF4005039
:100B800002904848006910B90220049001E0012059
:100B900004900220039005900320069002A9424889
:100BA00001F070F84FF48050029012200390012061
:100BB000049003200590069002A93B4801F062F8DA
:100BC0004FF400400290022003900590032006900D
:100BD00002A9354801F056F800220121242001F035
:100BE000DFF9242001F0C8F93048314908601020AD
:100BF000486000212E4881608021C1602948C0687A
:100C0000B0F5E06F04D8002129480161416105E099
:100C10004FF4807126480161890041610021244818
:100C200081614FF44051C16100F098FF00BF20483E
:100C30001C49C86408461E49486200BF08211C4878
:100C400000F07EFD002201210B2001F0A9F90B200C
:100C500001F092F917481349086000211148C16159
:100C60008160016141614FF4E061C1600021016276
:100C70004FF4802181614FF482700A49486000215D
:100C80000848816202F036F808B1FFF767FD0548B1
:100C900002F0E6F808B1FFF761FD07B000BD000003
:100CA00000100240AC65002000040048080002402B
:100CB000186600200038004000B587B000BF21480A
:100CC000406B40F004001F4948630846406B00F049
:100CD0000400019000BF00BF00BF0846406B40F019
:100CE000100048630846406B00F01000019000BF00
:100CF00000BF0120029000200390012004900220F8
:100D0000059002A94FF0904000F0BCFF4FF4005056
:100D1000029000200390012004900220059002A977
:100D2000094800F0AFFF802002900120039004905A
:100D30000220059002A94FF0904000F0A3FF07B0F9
:100D400000BD0000001002400008004800B587B058
:100D500000BF0D48406B40F008000B49486308464F
:100D6000406B00F00800019000BF00BF802002909F
:100D700001200390002004900220059002A903485E
:100D800000F080FF07B000BD0010024000040048E2
:100D900000B587B000BF2348406B40F004002149F4
:100DA00048630846406B00F00400019000BF00BF9C
:100DB000002209154FF0904001F050F800224FF446
:100DC00080714FF0904001F049F84FF4806002903C
:100DD00001200390002004900220059002A94FF00A
:100DE000904000F04FFF4FF480700290012003907C
:100DF000002004900220059002A94FF0904000F0DE
:100E000041FF00224FF480614FF0904001F026F83E
:100E100000224FF480714FF0904001F01FF807B0AE
:100E200000BD00000010024070B52DED068B054698
:100E30000024002006E0234A411C52F8211042F809
:100E40002010401C0728F6DB1E492868C8610846A8
:100E5000006898B30024002004E01A4951F82010DB
:100E60000C44401C0828F8DBE40800EE104AB8EEF9
:100E7000400AB0EE408A18EE100AFFF76BFA41EC18
:100E80001A0B9FED110B53EC102BFFF7F1F941EC0E
:100E9000190BFFF772FA08EE100AB0EE000A28EEFE
:100EA000000AB0EE408A9FED0A0AC8EE000AB0EED2
:100EB000608AB0EE480ABDEC068B70BDFFE79FED7F
:100EC000050AF8E78C6500200000000000000840DB
:100ED000000080450000000010B5014601200A68AE
:100EE00040F6B8339A420ED9094B1B78FF2B04DA2F
:100EF000074B1B785B1C064C2370054B1B780A2B99
:100F000005DD002003E00023014C2370012010BD0B
:100F10001500002010B520221449002002F0C1FF66
:100F20001248807F00041149497F40EA01200F499F
:100F3000097F08430E490860084600680D49884249
:100F400010D90D480068401C20B10B480068401CB7
:100F50000949086005200849086030B10E2003F0F7
:100F60004BF902E000200449086010BD9490002075
:100F700030640020CED604003864002010B5002272
:100F80004FF480614FF0904000F068FF00224FF472
:100F900080714FF0904000F061FF10BD10B501224C
:100FA00091024FF0904000F059FF012211024FF0E2
:100FB000904000F053FF10BDF8B504460026002015
:100FC000009000BF94F82800012801D10220F8BD4C
:100FD000012084F8280000BF2046FFF7DFFA06460C
:100FE000002E71D1E06A20F4885040F00200E062E7
:100FF000022001F03DF838490968B1FBF0F04000EB
:10100000009002E00098401E009000980028F9D15E
:101010002068806800F0010060B1E06A20F0020002
:1010200040F01000E06200BF002084F8280000BFFC
:101030000120CCE72068806840F0080021688860C3
:1010400000F012FF054611E000F00EFF401B0A28D9
:101050000CD9E06A20F0020040F01000E06200BF0E
:10106000002084F8280000BF0120B0E720688068D5
:1010700000F008000028E7D12068806840F00400F4
:101080002168886000F0F0FE054611E000F0ECFEFB
:10109000401B0A280CD9E06A20F0020040F0100042
:1010A000E06200BF002084F8280000BF01208EE726
:1010B0002068806800F004000028E7D1E06A20F092
:1010C000020040F00100E06200BF002084F8280028
:1010D00000BF30467BE700000000002038B5024624
:1010E00000230020009000BF92F82800012801D1C1
:1010F000022038BD012082F8280000BF4868072878
:1011000012D21068406B0C79641E04EB84051F2416
:10111000AC40A0430D796D1E05EB85050C68AC4015
:1011200020431468606327E048680D2812D21068D5
:10113000006B0C79E41F04EB84051F24AC40A04332
:101140000D79ED1F05EB85050C68AC402043146854
:10115000206311E01068C06A0C790D3C04EB840533
:101160001F24AC40A0430D790D3D05EB85050C68AF
:10117000AC4020431468E06208680A2812D3106863
:10118000C0680C780A3C04EB44050724AC40A0433B
:101190000D780A3D05EB45058C68AC40204314688A
:1011A000E0600FE0106800690C7804EB4405072448
:1011B000AC40A0430D7805EB45058C68AC4020435E
:1011C000146820610868102802D00868112827D107
:1011D000174C1068A0421ED11068806800F400000F
:1011E000F0B91068806840F400001468A0600868D6
:1011F000102815D10F4800680F4CB0FBF4F000EB3D
:1012000080004000009002E00098401E009000988E
:101210000028F9D104E0D06A40F02000D062012318
:1012200000BF002082F8280000BF184661E70000D8
:10123000002401400000002040420F0001460868E1
:10124000C06C70472DE9F0410446002700250026B8
:10125000A84614B90120BDE8F081E06808B9207EF5
:1012600000B100BF207E00B100BFE06A30B90020AD
:10127000206384F82800204600F09EF82046FFF7FF
:101280008DF90746E06A00F01000002878D1002FA1
:10129000FCD1E06A20F4885040F00200E062424A4B
:1012A000A1682068904208D1206AB0F5002F02D1D1
:1012B0004FF4002002E0206A00E0206A0143207C15
:1012C00041EA40000643E068B0F5807F02D0E06864
:1012D000012802D14FF4807000E0002061680843CB
:1012E0000543207E012811D1207C38B9E069401ED9
:1012F0004FF4006141EA4030054307E0E06A40F006
:101300002000E062206B40F001002063206840680C
:10131000264908402843216848602068806824499D
:101320000840304321688860E068B0F5807F02D0D3
:10133000E068012802D14FF4807000E00020B0F591
:10134000807F02D0207E012803D1A08A401E4FEA70
:1013500000582068C06A20F4700040EA0800216844
:10136000C8622068806813490840B04209D1002053
:101370002063E06A20F0020040F00100E06211E02A
:101380000BE0E06A20F0020040F01000E062206B09
:1013900040F001002063012704E0E06A40F0100003
:1013A000E0620127384656E7003C0140FF16FFFC8B
:1013B000FDF7E1FFFE0E1FFF10B586B004461421B5
:1013C00001A8FEF74AFF00BF2548806940F00100F0
:1013D000234988610846806900F00100009000BF41
:1013E00000BF00BF0846406940F001004861084660
:1013F000406900F00100009000BF00BF00BF084638
:10140000406B40F0040048630846406B00F0040065
:10141000009000BF00BF00BF0846406B40F00800CE
:1014200048630846406B00F00800009000BF00BF12
:1014300006200190032002900020039001A94FF0A4
:10144000904000F01FFC0220019003200290002039
:10145000039001A9034800F015FC06B010BD000080
:10146000001002400004004870B50446002500BF8B
:1014700094F82800012801D1022070BD012084F8D1
:10148000280000BF2046FFF7B3F80546002D77D1AE
:10149000E06A40F20121884340F48070E0623C49F8
:1014A0002068884208D13B48006800F4702008B9E1
:1014B000012002E0002000E0012078B1E06A20F481
:1014C0008010E0622068406800F4806000B3E06A49
:1014D00020F4005040F48050E06219E0E06A40F4EB
:1014E0008010E0622B49091F2068884203D02849F8
:1014F0002068884204D12748006800F4806000E03A
:10150000002028B1E06A20F4005040F48050E062EE
:10151000E06A00F4805020B1206B20F004002063CA
:1015200001E00020206300BF002084F8280000BFF5
:10153000C01E216808602068806800F46020B0F553
:10154000602F16D112492068884208D111480068DE
:1015500000F4702008B9012002E0002000E0012022
:1015600038B12068806840F4A000216888600CE0F1
:1015700006E02068806840F480102168886004E0FC
:1015800000BF002084F8280000BF284675E700004F
:10159000002801400424014070B50446002594F859
:1015A0002100022803D00420A0630125C1E02068A7
:1015B000006820F00E00216808602068006820F0B4
:1015C0000100216808605C492068884252D95A4964
:1015D00078392068884201D1012047E056496439B2
:1015E0002068884201D1102040E0534950392068DA
:1015F000884201D1801539E04F493C392068884242
:1016000001D1801432E04C4928392068884202D147
:101610004FF480302AE0484914392068884202D1CA
:101620004FF4801022E044492068884201D14004F0
:101630001CE042492068884201D1012016E03F4960
:1016400014312068884201D110200FE03B49283135
:101650002068884201D1801508E038493C31206873
:10166000884201D1801401E04FF480303349091FD2
:10167000086051E0304978392068884201D1012062
:1016800047E02D4964392068884201D1102040E0AC
:10169000294950392068884201D1801539E026490E
:1016A0003C392068884201D1801432E0224928392F
:1016B0002068884202D14FF480302AE01E49143954
:1016C0002068884202D14FF4801022E01A49206835
:1016D000884201D140041CE018492068884201D1A9
:1016E000012016E0154914312068884201D11020EC
:1016F0000FE0124928312068884201D1801508E0A6
:101700000E493C312068884201D1801401E04FF439
:101710008030094980394860012084F8210000BFE9
:10172000002084F8200000BF606B10B12046616B80
:101730008847284670BD000080000240080402402F
:1017400038B502461B4C1368A34206D21A4C1368E4
:101750001B1B1424B3FBF4F006E0164C13681B1B90
:101760001424B3FBF4F3D81D00BF144B9B6943F062
:101770000103124CA36123469B6903F0010300930C
:1017800000BF00BF022303EB90030D4C54F823303D
:101790008407E50E7F24AC40A3438407E40E01FADE
:1017A00004F42343022404EB9004054D45F824304F
:1017B00038BD00000804024008000240001002404A
:1017C0000000014070B50446E06B056820680668BB
:1017D00094F84010042088402840002875D006F076
:1017E00004000028FAD02068006800F0200028B922
:1017F0002068006820F0040021680860D54920684E
:10180000884254D9D34978392068884201D10420CC
:1018100049E0D04964392068884201D1402042E043
:10182000CC4950392068884201D100153BE0C949B4
:101830003C392068884202D14FF4804033E0C549EA
:1018400028392068884202D14FF480202BE0C1491A
:1018500014392068884202D14FF4800023E0BD494A
:101860002068884201D1C0041DE0BB49206888423D
:1018700001D1042017E0B84914312068884201D111
:10188000402010E0B44928312068884201D1001579
:1018900009E0B1493C312068884202D14FF48040D0
:1018A00001E04FF48020AC49091F086054E0A949C9
:1018B00078392068884201D104204AE0A54964397A
:1018C0002068884202D1402043E04CE0A1495039D1
:1018D0002068884201D100153BE09E493C392068D0
:1018E000884202D14FF4804033E09A492839206879
:1018F000884202D14FF480202BE0964914392068A9
:10190000884202D14FF4800023E092492068884247
:1019100001D1C0041DE090492068884201D1042013
:1019200017E08D4914312068884201D1402010E031
:10193000894928312068884201D1001509E086498B
:101940003C312068884202D14FF4804001E04FF4DE
:101950008020804980394860E06A002802D0204613
:10196000E16A8847F4E094F840100220884028405B
:10197000002871D006F002000028FAD02068006824
:1019800000F0200040B92068006820F00A002168BB
:101990000860012084F821006E492068884254D9EB
:1019A0006C4978392068884201D1022049E06949B0
:1019B00064392068884201D1202042E065495039CD
:1019C0002068884201D140153BE062493C392068DB
:1019D000884202D14FF4005033E05E492839206834
:1019E000884202D14FF400302BE05A491439206864
:1019F000884202D14FF4001023E056492068884203
:101A000001D180041DE054492068884201D10220A0
:101A100017E0514914312068884201D1202010E09C
:101A20004D4928312068884201D1401509E04A49D2
:101A30003C312068884202D14FF4005001E04FF45D
:101A400000304549091F086054E042497839206850
:101A5000884202D102204AE057E03E4964392068BA
:101A6000884201D1202042E03A495039206888421A
:101A700001D140153BE037493C392068884202D10A
:101A80004FF4005033E0334928392068884202D1AE
:101A90004FF400302BE02F4914392068884202D1DE
:101AA0004FF4001023E02B492068884201D18004C4
:101AB0001DE029492068884201D1022017E026490B
:101AC00014312068884201D1202010E022492831B9
:101AD0002068884201D1401509E01F493C31206847
:101AE000884202D14FF4005001E04FF40030194910
:101AF0008039486000BF002084F8200000BFA06A41
:101B000030B32046A16A884722E094F840100820AC
:101B100088402840E0B106F00800C8B1206800689D
:101B200020F00E002168086094F8401001208840E1
:101B3000E16B48600120A06384F8210000BF002011
:101B400084F8200000BF206B10B12046216B88472D
:101B500070BD0000800002400804024001460022DF
:101B600009B9012070471E4B086898420BD21D4BE3
:101B70000868C01A1423B0FBF3F080000864194809
:101B80000838C8630AE0164B0868C01A1423B0FB73
:101B9000F3F08000086412480838C863022081F816
:101BA00021000868026843F6F0708243D1E901031E
:101BB0001843CB6818430B6918434B6918438B696A
:101BC0001843CB6918430243086802600020886309
:101BD000012081F82100002081F8200000BFC1E72A
:101BE00008040240080002402DE9F04104460D4679
:101BF00016461F464FF0000800BF94F82000012849
:101C000002D10220BDE8F081012084F8200000BF4D
:101C100094F8210001282CD1022084F82100002012
:101C2000A0632068006820F00100216808603B463E
:101C3000324629462046FEF742FFE06A30B120686E
:101C4000006840F00E00216808600BE02068006822
:101C500020F00400216808602068006840F00A0055
:101C6000216808602068006840F001002168086071
:101C700006E000BF002084F8200000BF4FF00208FB
:101C80004046BFE778B503460022CAE001269640E9
:101C90000D6805EA0604002C71D04D68022D02D0B3
:101CA0004D68122D13D1D60803F1200555F82600F2
:101CB0005507EE0E0F25B540A8435607F60E0D69E1
:101CC000B5402843D60803F1200545F826001868DA
:101CD00056000325B540A8430D7905F003055600CD
:101CE000B540284318604D68012D08D04D68022D7D
:101CF00005D04D68112D02D04D68122D13D1986872
:101D000056000325B540A8435600CD68B54028438A
:101D10009860586801259540A8430D79C5F30015D2
:101D2000954028435860D86856000325B540A8431D
:101D300056008D68B5402843D8604D6805F0805541
:101D4000B5F1805F6CD100BF394DAD6945F001053B
:101D5000374EB5613546AD6905F00105009500BF08
:101D600000BF344D960855F8260095072E0F0F2515
:101D7000B540A843B3F1904F02D1002515E04FE0E4
:101D80002D4DAB4201D101250FE02C4DAB4201D1CD
:101D900002250AE02A4DAB4201D1032505E0294D79
:101DA000AB4201D1042500E007259607360FB54068
:101DB0002843204D960845F82600234D2868A04367
:101DC0004D6805F48035B5F5803F00D120431E4DA8
:101DD00028602D1D2868A0434D6805F40035B5F531
:101DE000003F00D12043184D2D1D28602D1D28686F
:101DF000A0434D6805F48015B5F5801F00D1204340
:101E0000114D083528602D1D2868A0434D6805F444
:101E10000015B5F5001F00D120430B4D0C3528608F
:101E2000521C0D68D540002D7FF430AF78BD000006
:101E3000001002401400014000040048000800485F
:101E4000000C0048001000480004014002461369DD
:101E50000B400BB1012000E0002070470AB1816106
:101E600000E0816270470000014800687047000090
:101E70004064002003480068034909780844014988
:101E800008607047406400204864002010B50420BA
:101E900000F0C4F8072000F005F800F04DF800202D
:101EA00010BD0000F0B587B00546002600270022CF
:101EB0002946362000F074F8362000F05DF800BFA7
:101EC0001948C06940F010001749C8610846C06948
:101ED00000F01000009000BF00BF01A902A800F0B0
:101EE000CBFB059E1EB900F0EFFB044602E000F0BC
:101EF000EBFB44000D48B4FBF0F0471E0C480D49C5
:101F0000086040F2E7310B48C16047600021016181
:101F10008160816101F0C2F820B9064801F0D9F86A
:101F200007B0F0BD0120FBE70010024040420F0067
:101F300000100040C464002008B500BF0D4880694F
:101F400040F001000B4988610846806900F00100FB
:101F5000009000BF00BF00BF0846C06940F080503D
:101F6000C8610846C06900F08050009000BF00BF03
:101F700008BD0000001002400146084600280DDBA5
:101F800000BF00BF00F01F0301229A4043099B00DD
:101F900003F1E023C3F8002100BF00BF00BF70477A
:101FA0002DE9F05F80460D461646002703F020F825
:101FB000074639462A46334601F00700C0F1070AB2
:101FC000BAF1030F02D94FF0030A01E0C0F1070A8A
:101FD000D14600F1030ABAF1070F02D24FF0000A0E
:101FE00001E0A0F1040AD4464FF0010A0AFA09FA06
:101FF000AAF1010A0AEA020A0AFA0CFA4FF0010BE6
:102000000BFA0CFBABF1010B0BEA030B4AEA0B04D6
:102010002146404602F0F4FFBDE8F09F00BF00F00B
:102020000702064B19684FF6FF031940044B0B4398
:1020300043EA0221014B196000BF70470CED00E03C
:102040000000FA0500BFBFF34F8F0748006800F497
:10205000E06006490843001D03490860BFF34F8F45
:1020600000BF00BF00BFFDE70CED00E00000FA0577
:102070002DE9F04F91B081464022A3A101A8FEF7BF
:10208000D3F8B1A000680090002600270024A046E5
:10209000A2460025A346B9F1010F09D0B9F1020FFC
:1020A0002DD0B9F1100F64D0B9F1200F70D1DCE060
:1020B000A648056A05F44070B0F5807F05D105F0AB
:1020C000020010B14FF4004B18E005F44070B0F579
:1020D000007F07D19D48406A00F0020010B149F628
:1020E000404B0BE005F44070B0F5407F06D19748B7
:1020F000006800F4003008B1DFF854B2FFE0934804
:10210000406894490840B0F5404F1FD007DC68B1E3
:10211000B0F5804F0FD0B0F5004F27D110E08E49B9
:102120000844C0B1B0F5004F20D11AE000F0DCFA4D
:102130004FEA500B1BE000F0D7FA4FEA900B16E085
:1021400000F0D2FA0621B0FBF1FB10E000F0CCFA6F
:102150004FEAD00B0BE000F0C7FA0C21B0FBF1FB0B
:1021600005E000F0C1FA4FEA101B00E000BF00BF1D
:10217000C5E07648856A05F00040B0F1004F08D10F
:102180007248806A00F0200018B1DFF8D0B16BE02F
:10219000B4E005F00040B0F1004F65D06B48006836
:1021A00000F0807000285FD06848466806F4701020
:1021B00006F0C04140EAD11001A901EB904090F82F
:1021C000008006F44030B0F5803F04D006F4403083
:1021D000B0F5403F0BD15D484068C0F340401DF86A
:1021E00000705F4808FB00F0B0FBF7F402E05D48C8
:1021F00008FB00F4554840685B4900EA010ABAF15F
:10220000000F16D009DCBAF1004F1FD057485044D8
:1022100000B3B0F5800F25D121E0BAF5800F06D0CC
:10222000BAF5000F0DD0BAF5400F1BD106E0A3465A
:1022300019E060000321B0FBF1FB14E04FEA540BFE
:1022400011E060000521B0FBF1FB0CE00320B4FBC2
:10225000F0FB08E060000721B0FBF1FB03E04FEA70
:10226000940B00E000BF00BF49E03848856B05F0E3
:102270000F00082803D005F0080008283DD005F01D
:102280000F00082807D13148006800F4003010B171
:10229000DFF8CCB031E02D48006800F0807060B30A
:1022A0002A48466806F4701006F0C04140EAD11092
:1022B00001A901EB904090F8008006F44030B0F5A1
:1022C000803F04D006F44030B0F5403F0BD11F48AA
:1022D0004068C0F340401DF80070214808FB00F042
:1022E000B0FBF7F402E01F4808FB00F41748806BCE
:1022F00000F00F00401CB4FBF0FB00E000BF00BF8B
:10230000584611B0BDE8F08F02030405060708091E
:102310000A0B0C0D0E0F10111213141516171819A5
:102320001A1B1C1D1E1F2021222324252627282995
:102330002A2B2C2D2E2F3031323334353637383985
:102340003A3B3C3D3E3F3F3F01020000001002404F
:102350006CDC020000C0001000C0FFEF006CDC026B
:1023600000366E0100127A000000C0800000C07FBD
:10237000F8B5044600260025207800F0010000286A
:1023800071D000275548C06900F0805070B900BF77
:102390005248C06940F080505049C8610846C06941
:1023A00000F08050009000BF00BF01274C4800683B
:1023B00000F48070B0B94A48006840F48070484921
:1023C0000860FFF751FD064606E0FFF74DFD801B54
:1023D000642801D90320F8BD4148006800F48070EA
:1023E0000028F2D03D48006A00F440755DB3A08833
:1023F00000F44070A84226D03848006A20F44075A6
:102400003648006A40F48030344908620846006A61
:1024100020F4803008620846056205F0010090B1A2
:10242000FFF722FD064608E0FFF71EFD801B41F284
:102430008831884201D90320CDE72848006AC0F3DB
:1024400040000028F0D02548006A20F44070616800
:10245000084322490862012F04D10846C06920F0D0
:102460008050C86100BF207800F00200022807D128
:102470001A4840681B490840A1680843174948604A
:10248000207800F01000102818D1E068B0F1004F5B
:102490000ED01248806A20F0004010498862084639
:1024A000406811490840E16808430C49486005E06C
:1024B0000A48806A40F0004008498862207800F0AD
:1024C0002000202807D10548806B20F00F002169EB
:1024D00008430249886300207DE7000000100240A5
:1024E00000700040FF3FFFEFFFFF3F7F70B50446E5
:1024F0000D460CB9012070BD5A48006800F00F006D
:10250000A8420ED25748006820F00F0028435549D2
:1025100008600846006800F00F00A84201D00120C2
:10252000E9E7207800F0020002281DD1207800F0B1
:102530000400042805D14C48406840F4E0604A4952
:102540004860207800F00800082805D14648406817
:1025500040F46050444948604348406820F0F0002F
:10256000A168084340494860207800F0010078B332
:102570006068012806D13C480068C0F3404090B92B
:102580000120B8E76068022806D13748006800F0EB
:10259000807040B90120AEE733480068C0F34000C6
:1025A00008B90120A7E73048406820F003006168BF
:1025B00008432D494860FFF757FC064609E0FFF73E
:1025C00053FC801B41F28831884202D9032092E7F4
:1025D00007E02548406800F00C006168B0EB810F0F
:1025E000EDD12048006800F00F00A8420ED91D4828
:1025F000006820F00F0028431A4908600846006868
:1026000000F00F00A84201D0012074E7207800F00C
:102610000400042807D11448406820F4E060E16811
:10262000084311494860207800F00800082808D1C4
:102630000D48406820F46050216940EAC1000A4911
:10264000486000F061F808494968C1F30311074A7E
:10265000515CC8400649086006480068FFF722FC44
:10266000002048E70020024000100240B46E00083D
:1026700000000020446400200F2202600D4A5268CE
:1026800002F0030242600B4A526802F0F0028260DC
:10269000084A526802F4E062C260064A526802F4D4
:1026A0006052D2080261044A126802F00F020A6006
:1026B00070470000001002400020024001480068FE
:1026C000704700000000002000B5FFF7F7FF044945
:1026D0004968C1F30221034A515CC84000BD0000B3
:1026E00000100240C46E000800B5FFF7E7FF044980
:1026F0004968C1F3C221034A515CC84000BD0000D3
:1027000000100240C46E00082DE9F04192B0402252
:1027100022A102A8FDF788FD30A0006801900024E6
:10272000002500260027A0462D48446804F00C0030
:1027300060B3042802D0082827D102E0DFF8A48083
:1027400027E004F4701004F0C04140EAD11002A95F
:1027500001EB9040077804F44030B0F5803F04D09E
:1027600004F44030B0F5403F0AD11D484068C0F342
:10277000404001A90D5C1B487843B0FBF5F602E030
:10278000194807FB00F6B04603E000BFDFF85880A9
:1027900000BF00BF404612B0BDE8F081020304054F
:1027A000060708090A0B0C0D0E0F10111213141551
:1027B000161718191A1B1C1D1E1F20212223242541
:1027C000262728292A2B2C2D2E2F30313233343531
:1027D000363738393A3B3C3D3E3F3F3F010200002F
:1027E0000010024000366E0100127A00F8B504466F
:1027F0000CB90120F8BD207800F00100002873D04A
:10280000F748406800F00C00042813D0F4484068F2
:1028100000F00C00082818D1F148406800F480301E
:10282000B0F5803F06D0EE48406800F48030B0F547
:10283000403F0AD1EA480068C0F3404000286CD00D
:102840006068002869D10120D4E76068B0F5803F56
:1028500007D1E348806B20F44070A1680843E04949
:10286000886300BF6068B0F5803F06D1DC4800682F
:1028700040F48030DA49086028E0606858B9D848E8
:10288000006820F48030D64908600846006820F4CB
:10289000802008601AE06068B0F5A02F0BD1D04806
:1028A000006840F48020CE4908600846006840F483
:1028B000803008600AE0CA48006820F48030C849C7
:1028C00008600846006820F48020086000BF606847
:1028D00090B1FFF7C9FA054607E0FFF7C5FA401BBC
:1028E000642802D9032085E717E0BD480068C0F3DB
:1028F00040400028F1D010E0FFF7B6FA054606E0A8
:10290000FFF7B2FA401B642801D9032072E7B448EC
:102910000068C0F340400028F2D1207800F00200A7
:10292000022854D1AE48406800F00C0098B1AC4881
:10293000406800F00C00082817D1A948406800F44E
:102940008030B0F5803F10D0A548406800F480305A
:10295000B0F5403F09D0A2480068C0F3400078B30A
:102960006069012833D0012044E76069B8B19C4810
:10297000006840F001009A490860FFF775FA0546C3
:1029800006E0FFF771FA401B022801D9032031E766
:1029900093480068C0F340000028F2D017E0904848
:1029A000006820F001008E490860FFF75DFA0546D7
:1029B00007E0FFF759FA401B022802D9032019E764
:1029C00005E087480068C0F340000028F1D1207876
:1029D00000F01000102830D1A069B8B18048806A9A
:1029E00040F010007E498862FFF73EFA054606E097
:1029F000FFF73AFA401B022801D90320FAE678488B
:102A0000806AC0F340100028F2D016E07448806A53
:102A100020F0100072498862FFF726FA054606E0AA
:102A2000FFF722FA401B022801D90320E2E66C4896
:102A3000806AC0F340100028F2D1207800F008002E
:102A4000082833D1E069D0B16548406A40F0010000
:102A500063494862FFF708FA054606E0FFF704FA03
:102A6000401B022801D90320C4E65D48406AC0F338
:102A700040000028F2D0012001F024FA16E0584866
:102A8000406A20F0010056494862FFF7EDF905461B
:102A900006E0FFF7E9F9401B022801D90320A9E667
:102AA0004F48406AC0F340000028F2D1207800F07F
:102AB0000400042875D100274948C06900F08050FF
:102AC00070B900BF4648C06940F080504449C861B1
:102AD0000846C06900F08050009000BF00BF012789
:102AE0004048006800F48070B0B93E48006840F487
:102AF00080703C490860FFF7B7F9054606E0FFF72C
:102B0000B3F9401B642801D9032073E635480068F7
:102B100000F480700028F2D0E068012807D1304826
:102B2000006A20F01800216908432D49086200BF9F
:102B3000E068012806D12A48006A40F001002849CF
:102B4000086227E0E06858B92548006A20F00100D3
:102B5000234908620846006A20F00400086219E070
:102B6000E06805280BD11E48006A40F004001C49AB
:102B700008620846006A40F0010008620AE018484E
:102B8000006A20F00100164908620846006A20F039
:102B90000400086200BFE068A0B1FFF765F90546D0
:102BA00009E030E0FFF760F9401B41F288318842CC
:102BB00001D903201EE60A48006AC0F3400000283D
:102BC000F0D017E0FFF750F905460DE0FFF74CF99C
:102BD000401B41F28831884206D903200AE60000F2
:102BE00000100240007000403F48006AC0F34000FF
:102BF0000028EBD1012F05D13B48C06920F080505F
:102C00003949C86100BF206A90B33748406800F076
:102C10000C00082853D0206A022838D132480068B6
:102C200020F0807030490860FFF71EF9054606E085
:102C3000FFF71AF9401B022801D90320DAE52A48D8
:102C40000068C0F340600028F2D1D4E909010843CC
:102C500025494968254A11400843234948600846E8
:102C6000006840F080700860FFF7FEF8054607E056
:102C700037E0FFF7F9F8401B022801D90320B9E536
:102C800019480068C0F340600028F2D029E01648D7
:102C9000006820F0807014490860FFF7E5F80546E9
:102CA00006E0FFF7E1F8401B022801D90320A1E567
:102CB0000D480068C0F340600028F2D111E0206A9E
:102CC000012800D196E50848466806F48031606A1C
:102CD000814204D106483040A16A884201D00120D7
:102CE00088E5002086E5000000100240FFFFC09F3D
:102CF00000003C6010B504460CB9012010BD022054
:102D000084F855002068006820F0400021680860C1
:102D1000204600F017F90020A06584F8550000BF98
:102D200084F8540000BF00BFE8E77047F8B50446D8
:102D30002068466820688568C5F3801048B905F0AA
:102D4000010030B1C6F3801018B12046616C88478D
:102D5000F8BDC5F3400030B1C6F3C01018B120462D
:102D6000A16C8847F4E7C5F3401018B9C5F380108B
:102D7000002871D0C6F3401000286DD0C5F3801034
:102D8000F0B194F8550003280ED0A06D40F0040077
:102D9000A06500BF002000902068C06800902068F7
:102DA0008068009000BF0BE000BF0020009020680A
:102DB000C068009020688068009000BF00BFC7E72F
:102DC000C5F3401088B1A06D40F00100A06500BFC0
:102DD000002000902068806800902068006820F043
:102DE00040002168086000BF00BFA06D70B320687C
:102DF000406820F0E00021684860012084F8550018
:102E000006F0020010B906F0010000B32068406827
:102E100020F0030021684860206D50B10F48216DFB
:102E20004863206DFEF7B8FB18B1A06D40F040007C
:102E3000A065E06C50B10948E16C4863E06CFEF7B6
:102E4000ABFB18B1A06D40F04000A06502E0204649
:102E5000FFF76BFF7CE7FFE700BF79E7FD3E000867
:102E600070B504460CB9012070BD6068B0F5827F72
:102E700000D101E00021E1610021A16294F8550038
:102E800028B9002084F85400204600F05CF80220A5
:102E900084F855002068006820F040002168086030
:102EA000E068B0F5E06F01D9002501E04FF48055EE
:102EB000E068B0F5706F05D0E068B0F5E06F01D064
:102EC0000021A162A08800F48270218901F40441EC
:102ED0000843217C01F002010843217D01F001013A
:102EE0000843218B01F400710843217F01F0380170
:102EF0000843A18901F4006108432021095D01F024
:102F000080010843218D01F40051084321680860C5
:102F10000421A06901EA1040A18C01F4004108439A
:102F200005F480510843216848602068C06920F496
:102F300000602168C8610020A065012084F8550068
:102F4000002091E7704770472DE9F04104460E4696
:102F50001546002700BF94F85400012802D1022032
:102F6000BDE8F081012084F8540000BF94F85500BA
:102F7000012801D0022780E006B10DB901277CE0CD
:102F8000032084F855000020A0652663A586E58609
:102F9000A063A0646064A087E087A068B0F5004FDC
:102FA0000BD12068006820F040002168086020688C
:102FB000006840F48040216808603348E16CC862D2
:102FC0003248E16C88623248E16C08630020E16CB1
:102FD00048632068406820F4804021684860E068C9
:102FE000B0F5E06F1DD8E06C4069B0F5806F18D186
:102FF000E08E00F0010048B92068406820F480406D
:1030000021684860E08E4010E0860AE02068406851
:1030100040F4804021684860E08E012101EB6000AF
:10302000E086E38ED4F800C00CF10C02216BE06C5A
:10303000FEF7DAFD40B1A06D40F01000A065012759
:10304000012084F8550018E02068006800F0400076
:10305000402805D02068006840F0400021680860E2
:103060002068406840F0200021684860206840687F
:1030700040F002002168486000BF00BF002084F8D3
:10308000540000BF38466BE7393F0008473F00084F
:10309000113F0008704770477047704710B50446ED
:1030A0000CB9012010BD94F83D0028B9002084F827
:1030B0003C00204600F00CF8022084F83D00211D61
:1030C000206801F0F1FA012084F83D000020E9E7D2
:1030D000704701460868C06840F001000B68D8607E
:1030E0000868806800F00702062A05D008680068B2
:1030F00040F001000B68186000207047704710B561
:10310000044620680069C0F34000D8B12068C06858
:10311000C0F34000B0B16FF00200216808610120E7
:1031200020772068806900F0030018B12046FFF77F
:10313000E5FF05E0204600F0ADF8204600F0AEF9CE
:103140000020207720680069C0F38000D8B1206893
:10315000C068C0F38000B0B16FF00400216808615E
:10316000022020772068806900F4407018B1204662
:10317000FFF7C4FF05E0204600F08CF8204600F081
:103180008DF90020207720680069C0F3C000D8B115
:103190002068C068C0F3C000B0B16FF008002168BB
:1031A0000861042020772068C06900F0030018B18E
:1031B0002046FFF7A3FF05E0204600F06BF820460D
:1031C00000F06CF90020207720680069C0F300103F
:1031D000D8B12068C068C0F30010B0B16FF0100023
:1031E00021680861082020772068C06900F44070D9
:1031F00018B12046FFF782FF05E0204600F04AF8AC
:10320000204600F04BF9002020772068006900F08C
:10321000010058B12068C06800F0010030B16FF0C3
:10322000010021680861204600F0AAF920680069C1
:10323000C0F3C01058B12068C068C0F3C01030B1EE
:103240006FF08000216808612046FFF725FF2068A5
:103250000069C0F3801058B12068C068C0F38010C6
:1032600030B16FF0400021680861204600F08DF910
:1032700020680069C0F3401058B12068C068C0F3EE
:10328000401030B16FF02000216808612046FFF740
:1032900004FF10BD704770B504460D46164600BFCA
:1032A00094F83C00012801D1022070BD012084F86F
:1032B0003C0000BF022084F83D0036B1042E1BD034
:1032C000082E31D00C2E5ED145E02946206801F051
:1032D00069FA2068806940F00800216888612068E8
:1032E000806920F00400216888612068806929696C
:1032F00008432168886147E02946206801F08AFA7E
:103300002068806940F400602168886120688069D5
:1033100020F480602168886120688069296940EA1A
:103320000120216888612FE02946206801F0B0FA69
:103330002068C06940F008002168C8612068C06941
:1033400020F004002168C8612068C0692969084329
:103350002168C86118E02946206801F0D5FA206884
:10336000C06940F400602168C8612068C06920F429
:1033700080602168C8612068C069296940EA01202D
:103380002168C86100E000BF00BF012084F83D0053
:1033900000BF002084F83C0000BF00BF85E710B5E7
:1033A00004460CB9012010BD94F83D0028B9002056
:1033B00084F83C00204600F00DF8022084F83D001F
:1033C000211D206801F070F9012084F83D000020E3
:1033D000E9E7000010B586B00446142101A8FCF707
:1033E0003CFF00BF2B48806940F400602949886198
:1033F0000846806900F40060009000BF00BF00BF75
:103400000846C06940F00200C8610846C06900F083
:103410000200009000BF00BF00BF0846406B40F0B4
:10342000040048630846406B00F00400009000BFB1
:1034300000BF00BF0846406B40F0080048630846E4
:10344000406B00F00800009000BF00BF0220029017
:1034500001200390022004900002019004200590B6
:1034600001A94FF09040FEF70DFC012001900620CD
:10347000059001A90848FEF705FC082001900120ED
:10348000029003900220049001A90348FEF7FAFB82
:1034900006B010BD00100240000400487047000054
:1034A00070B504460E4601223146206801F068F9E5
:1034B0000F492068884203D00E492068884201D114
:1034C000012000E0002028B12068406C40F400405A
:1034D000216848642068806800F00705062D05D043
:1034E0002068006840F0010021680860002070BD7D
:1034F000002C01400034014030B504460D46002246
:103500002946206801F03CF91B492068884203D015
:103510001A492068884201D1012000E0002090B1C2
:1035200000BF2068006A41F21111084050B92068BC
:10353000006A8910084028B92068406C20F40040D7
:103540002168486400BF00BF2068006A41F2111181
:10355000084050B92068006A8910084028B92068DE
:10356000006820F001002168086000BF012084F895
:103570003D00002030BD0000002C0140003401401F
:1035800010B50446FEF776FC10BD704710B5044632
:103590000CB9012010BDA06900B100E000BF94F893
:1035A000450028B9002084F84400204600F02CF89B
:1035B000242084F845002068C06820F40050216869
:1035C000C860204601F0EEFA206A10B1204601F0F2
:1035D000CFFA2068006920F49040216808612068D3
:1035E000406920F02A00216848612068C06840F4E2
:1035F00000502168C8600020A064202084F84500A5
:1036000084F846000020C5E770472DE9F84F0446CE
:103610000D46174699464FF0000A94F845002028B9
:1036200064D105B117B90120BDE8F88FA068B0F5E5
:10363000805F06D1206920B905F0010008B10120A2
:10364000F2E700BF94F84400012801D10220EBE723
:10365000012084F8440000BF0020A064212084F8E9
:103660004500FEF701FC824627866786A068B0F514
:10367000805F04D1206910B90026A84602E02E46DA
:103680004FF000081BE05346002280212046CDF871
:10369000009001F015FC08B10320C5E746B9B8F861
:1036A0000000C0F308002168486008F1020803E048
:1036B000307821684860761C608E401E6086608E7F
:1036C0000028E0D15346002240212046CDF800904A
:1036D00001F0F6FB08B10320A6E7202084F845009E
:1036E00000BF002084F8440000BF9DE702209BE754
:1036F00000BFFEE710B500224FF480710E48FEF7C0
:10370000ADFB01F055FC00224FF400710A48FEF7B2
:10371000A5FB022000F012F8012211020648FEF774
:103720009DFB022000F00AF800224FF4807102484D
:10373000FEF794FB10BD000000040048014601E0C4
:103740004A1E91B20029FBDC7047000010B5002230
:103750004FF480710D48FEF781FB01F029FC012236
:1037600051020A48FEF77AFB0220FFF7E7FF012229
:1037700011020648FEF772FB0220FFF7DFFF00226E
:103780004FF480710148FEF769FB10BD000400484A
:1037900070B505460826002401F0F4FB1AE0600627
:1037A000040E00224FF480711148FEF757FB0220EF
:1037B000FFF7C4FF012211020D48FEF74FFB022064
:1037C000FFF7BCFF4FF400710948FEF73FFB08B15B
:1037D00044F00104301EA6F10101CEB2DFD115B1D3
:1037E000FFF7B4FF01E0FFF785FF204670BD000042
:1037F000000400482DE9F05F0746884691461E46C2
:10380000DDE90AAB00F042F8384600F0D3F805468F
:1038100025B100F061F80120BDE8F09F404600F0BE
:10382000C9F805461DB100F057F80220F4E7BBF1D6
:10383000000F08D0484600F0BDF805461DB100F065
:103840004BF80320E8E700F021F8791CC8B200F03B
:10385000B1F805461DB100F03FF80420DCE7002474
:103860000EE0AAF10100A04204DD0020FFF790FF66
:10387000305503E00120FFF78BFF3055601CC4B2C8
:103880005445EEDB00F028F80020C5E710B501F044
:103890008FFB012211020F48FEF7E0FA01225102CC
:1038A0000C48FEF7DBFA0220FFF748FF00224FF436
:1038B00000710848FEF7D2FA0520FFF73FFF00220B
:1038C0004FF480710348FEF7C9FA0220FFF736FF74
:1038D000002010BD0004004810B500224FF4807194
:1038E0000F48FEF7BBFA00224FF400710C48FEF7B8
:1038F000B5FA01F05DFB0220FFF720FF0122110263
:103900000748FEF7ABFA0520FFF718FF0122510226
:103910000348FEF7A3FA0220FFF710FF10BD0000D6
:103920000004004810B5002400224FF480711A48AA
:10393000FEF794FA00224FF400711748FEF78EFA52
:1039400001F020FB0220FFF7F9FE012211021248CC
:10395000FEF784FA0220FFF7F1FE0BE0601C84B250
:10396000B4F57A7F06DDFFF7B7FF0CA001F038FB56
:10397000012010BD4FF400710748FEF767FA0028D8
:10398000ECD100224FF480710348FEF767FA01F092
:103990000FFB0020EDE70000000400484949435FA9
:1039A0005761697441636B2054494D454F55540D1F
:1039B0000A00000070B50446082501F0F9FA21E07C
:1039C00000224FF480711448FEF748FA04F080009A
:1039D00028B1012251021048FEF740FA05E000220A
:1039E0004FF400710C48FEF739FA6006040E02200D
:1039F000FFF7A4FE012211020748FEF72FFA02206A
:103A0000FFF79CFE281EA5F10101CDB2D8D1FFF72A
:103A100089FF0646304670BD000400482DE9F0419C
:103A200080460E461746FFF731FF4046FFF7C2FFBC
:103A3000054665B9002407E0305DFFF7BBFF05468A
:103A400005B103E0601C84B2BC42F5DB00BFFFF7A8
:103A500043FF2846BDE8F08110B504469F230022AD
:103A60004F21104602F0F8FA00224FF48051094825
:103A7000FEF7F4F94FF4C84221460748FFF764FA0D
:103A80004FF47A7001F0F0FA012211030148FEF7B9
:103A9000E5F910BD00040048AC65002070B505468E
:103AA0000C461646234622462946284602F0D4FAFA
:103AB00000224FF480510648FEF7D0F9304600F05E
:103AC00070F8012211030248FEF7C8F970BD00002A
:103AD0000004004838B5044620128DF80000E0B21A
:103AE0008DF8010000200CE09DF80010084A02F853
:103AF00010109DF80110012202EB4002044B995472
:103B0000401CB0F5485FEFDB0148FFF7A5FF38BD6B
:103B10003000002000B587B000BF1048406B40F077
:103B200008000E4948630846406B00F00800019009
:103B300000BF00BF081502900120039000200490F0
:103B40000220059002A90648FEF79CF800224FF4D7
:103B500080610348FEF782F907B000BD0010024003
:103B6000000400482DE9F04105460F4614469846EA
:103B700009E02678434632463946284601F084FA61
:103B8000A81DC5B2641C20780028F2D1BDE8F081E0
:103B900038B504468DF800400121684600F024F84D
:103BA00038BD38B5044620128DF80000E0B28DF81B
:103BB00001000221684600F017F838BD38B5044608
:103BC000009400224FF480410648FEF747F9012196
:103BD000684600F009F8012291030248FEF73EF919
:103BE00038BD00000004004870B504460D460022B0
:103BF0004FF480510648FEF731F92A462146054820
:103C0000FFF7A2F9012211030148FEF727F970BD61
:103C100000040048AC65002000BFFEE770B5044614
:103C20000D462D482D49086063212C48C1602C4861
:103C3000B0FBF4F0401E294948600021274801618B
:103C4000816041618161FFF7AAFB08B1FCF786FD45
:103C50006020244908600020886008610820C8604E
:103C60000020886148610846456004221B48FFF730
:103C700012FB08B1FCF772FD1B481C490860632168
:103C80001A48C1601648B0FBF4F0401E174948605E
:103C9000002116480161816041618161FFF77FFB6E
:103CA00008B1FCF75BFD31201049096848626020CB
:103CB0000F4908600020886008610820C860002063
:103CC000886148610846456008220848FFF7E3FA22
:103CD00008B1FCF743FD70BD002C0140A066002038
:103CE00000A60E002067002000040040E0660020CF
:103CF0003C67002070472DE9F04104460D4616460A
:103D00000027324629462046FFF788FE07463846F8
:103D1000BDE8F08130B585B08821502000F0AFF8C3
:103D200004464FF4FA70FFF709FD4FF4FA70FFF7FD
:103D300005FD4FF4FA70FFF701FD4FF4FA70FFF73D
:103D4000FDFC4FF4FA70FFF7F9FC4FF4FA70FFF73F
:103D5000F5FC4FF4FA70FFF7F1FC4FF4FA70FFF73F
:103D6000EDFC4FF4FA70FFF7E9FC4FF4FA70FFF73F
:103D7000E5FC4FF4FA70FFF7E1FC4FF4FA70FFF73F
:103D8000DDFC3CB940F223252A463349502000F09F
:103D900067F8044634B936252A4630495020FFF7E3
:103DA000AAFF04464FF4FA70FFF7C8FC4FF4FA700C
:103DB000FFF7C4FC4FF4FA70FFF7C0FC4FF4FA7041
:103DC000FFF7BCFC4FF4FA70FFF7B8FC4FF4FA7041
:103DD000FFF7B4FC4FF4FA70FFF7B0FC4FF4FA7041
:103DE000FFF7ACFC4FF4FA70FFF7A8FC4FF4FA7041
:103DF000FFF7A4FC4FF4FA70FFF7A0FC4FF4FA7041
:103E0000FFF79CFC54B901200A2102AB0022CDE946
:103E1000001020215020FFF7EDFC04464FF4FA700B
:103E2000FFF78CFC54B901200A2102ABC022CDE976
:103E3000001023215020FFF7DDFC04468A2150208A
:103E400000F01DF804468C21502000F018F80446BC
:103E5000204605B030BD00001A7300083D7500080B
:103E60002DE9F04104460D46164600273246294604
:103E70002046FFF7D3FD07463846BDE8F08170B510
:103E800006460C46FFF702FD3046FFF793FD054658
:103E90001DB92046FFF78EFD0546FFF71DFD28469C
:103EA00070BD7CB504460D4616460020CDE9006085
:103EB00004F03F0040F040012B4600225020FFF765
:103EC00099FC7CBD08B508490968C9084FF47A72A5
:103ED000B1FBF2F14143009100BF00BF00994A1EBF
:103EE00000920029F9D108BD0000002010B5024859
:103EF000FEF71CFF10BD0000AC65002070B5054644
:103F00006C6A0020E087E0862046FEF70EFF70BD59
:103F100070B505466C6A2068406820F0030021688F
:103F20004860A06D40F01000A065012084F85500A5
:103F30002046FEF7FAFE70BD70B50446656A284655
:103F4000FFF7A9F870BDF8B505466C6AFDF78CFF60
:103F500006462868006800F0200020282DD0206840
:103F6000406820F02000216848602068406820F008
:103F700002002168486032466421204600F022F8A1
:103F800018B1A06D40F02000A065A06850B900BF36
:103F9000002000902068C068009020688068009031
:103FA00000BF00BF0020E086012084F85500A06D0E
:103FB00018B12046FEF7B9FEF8BD2046FFF76AF8B3
:103FC00000BFF9E7F8B504460E4615463346002211
:103FD0004FF4C0512046009500F026F828B1A06D9E
:103FE00040F02000A0650320F8BD33460022802168
:103FF0002046009500F094F828B1A06D40F0200014
:10400000A0650320F0E7334600224FF4C06120464C
:10401000009500F009F828B1A06D40F02000A065DF
:104020000320E1E70020DFE72DE9FC5F04460D46B1
:1040300016461F46DDF8309000200090FDF714FF73
:10404000A0EB0900A7EB0008FDF70EFF82462068F1
:1040500000F10C0B31480068C0EBC00000EB8000A1
:10406000000D00FB08F0019050E0B5F5C06F05D1E0
:1040700026B99BF8000000909DF80000781C0028ED
:1040800044D0FDF7F1FEA0EB0A00404502D2B8F1A2
:10409000000F34D12068406820F0E00021684860BB
:1040A0006068B0F5827F0DD1A068B0F5004F03D0F5
:1040B000A068B0F5806F05D12068006820F040004E
:1040C00021680860A06AB0F5005F0DD100BF2068CC
:1040D000006820F40050216808602068006840F4FF
:1040E00000502168086000BF012084F8550000BF1F
:1040F000002084F8540000BF0320BDE8FC9F019815
:1041000008B94FF000080198401E019020688068AF
:104110002840B042A9D10020EFE7000000000020B5
:104120002DE9F84F04460D4690461E46DDF82890CE
:10413000FDF79AFEA0EB0900371AFDF795FE8246BF
:104140002C480068C0F3CB307843009045E0701CE9
:10415000002842D0FDF788FEA0EB0A00B84200D24A
:10416000A7BB2068406820F0E000216848606068D4
:10417000B0F5827F0DD1A068B0F5004F03D0A068E4
:10418000B0F5806F05D12068006820F040002168FC
:104190000860A06AB0F5005F0DD100BF206800681C
:1041A00020F40050216808602068006840F4005046
:1041B0002168086000BF012084F8550000BF00207E
:1041C00084F8540000BF0320BDE8F88FFFE7009893
:1041D00000B900270098401E0090206880682840A1
:1041E000A84201D1012000E000204045AFD10020CD
:1041F000EAE700000000002038B5044600940023E0
:104200005A1E69460248006802F0A2F938BD000053
:104210000400002038B50446009400231A4669467D
:104220000248006802F038FA38BD0000040000209F
:1042300038B50446009400235A1E694602480068B7
:1042400002F086F938BD00000800002010B50446D1
:1042500034B1012C08D0022C0BD0032C12D10DE06C
:10426000002001F04FFD0EE04FF47F0001F04AFD09
:1042700009E04FF47F4001F045FD04E0FF2001F02C
:1042800041FD00E000BF00BF10BD000070B5044656
:104290000D46012208210B48FDF7E0FD690860008A
:1042A000FFF7BCFC04210848FFF7FAF808B1FCF757
:1042B00055FA08210548FFF7F3F808B1FCF74EFA64
:1042C00070BD000000040048A0660020E0660020E9
:1042D00008B50027002600BF00BF64226946C64813
:1042E000006802F033FA0746012F73D19DF80000F1
:1042F000801E11286FD2DFE800F009296E6E5C3D48
:10430000C8C3F1F0F5FF2C30EDECEB00761C0A2071
:10431000B6FBF0F100FB116010B90320FFF76CFF52
:10432000B648006920B1B5480069401EB34908612C
:10433000B2480069012808D1B048007D28B90A2098
:10434000FFF75AFF0120FFF773FF4FE1FCF7E2FD93
:104350004CE10F20FFF750FF48E1A848006940B941
:104360006420A64908610B20FFF746FF0220FFF7F3
:104370005FFF3BE141F28830A049C8600846007801
:1043800050B9012008700820886041F28830C86068
:104390001220FFF731FF0BE098480078012807D181
:1043A00000F04AF91020FFF727FF0020FFF740FF39
:1043B0001CE141F288309149C86008460078012824
:1043C0002FD108464068062806D208464068401C9F
:1043D000486006E00BE108E10320884948600820B6
:1043E000886086484068032806D0042808D005283D
:1043F0000BD0062813D10DE01F20FFF76BFB0FE059
:104400004FF61F00FFF766FB0AE04FF6E070FFF77C
:1044100061FB05E040F2FF70FFF75CFB00E000BFCE
:104420002DE076480078022829D174488068092850
:1044300005D272488068401C7049886002E00720FD
:104440006E4988606D488068072804D0082807D026
:1044500009280FD109E047F6FF70FFF73BFB0AE0A0
:104460004FF6E070FFF736FB05E04BF64040FFF7F4
:1044700031FB00E000BF00BF0C20FFF7BDFEB5E040
:1044800041F288305D49C860B0E041F288305B4954
:10449000C86008460078012805D1022008700C2069
:1044A000FFF7AAFE09E055480078022805D101204F
:1044B000524908700D20FFF79FFE504840680328BE
:1044C0000DD14E480078022809D1FCF767FD08E0BD
:1044D00086E080E07BE00FE004E075E016E0FCF7AA
:1044E0004DFD83E00020454908750A20FFF784FE52
:1044F0000120FFF79DFE79E00120404908750B205F
:10450000FFF77AFE0020FFF793FE6FE03B4840681C
:10451000032806D0042817D0052828D006284CD117
:1045200038E0A02535488068072801D11E240AE01C
:1045300032488068082801D1282404E02F48806888
:10454000092800D1322439E0A0252C4880680728AA
:1045500001D11E240AE029488068082801D12824B6
:1045600004E026488068092800D1322426E0A025EE
:1045700022488068072801D11E240AE01F4880686D
:10458000082801D1282404E01C488068092800D1AB
:10459000322413E0A02519488068072801D11E2481
:1045A0000AE016488068082801D1282404E013484E
:1045B0008068092800D1322400E000BF00BF2146F6
:1045C0002846FFF763FE11E000F01AF80EE0002025
:1045D000FFF780FA0AE04FF47840FFF77BFA05E036
:1045E00040F2FF70FFF776FA00E000BF00BF022044
:1045F00001F024FE71E600000400002018000020F5
:1046000010B5002208210948FDF728FC04210848BC
:10461000FEF772FF08B1FCF7A1F808210548FEF784
:104620006BFF08B1FCF79AF810BD000000040048C9
:10463000A0660020E06600200020054908700320E5
:1046400048600820886041F28830C86070470000E8
:104650001800002010B502F05FF9012801D001F028
:10466000E7FE10BD10B5FCF77FF80648006840F47F
:104670007000044908604FF000600249803908600A
:1046800010BD000088ED00E010B50248FEF737FDD0
:1046900010BD0000A066002010B50248FEF72FFDF7
:1046A00010BD0000C464002010B50268294B984278
:1046B0000ED0B0F1804F0BD0274B984208D0274B3B
:1046C000984205D0264B984202D0264B984203D1FF
:1046D00022F070024B681A431E4B984220D0B0F172
:1046E000804F1DD01C4B98421AD01C4B984217D0BB
:1046F0001B4B984214D01B4B984211D01A4B984236
:104700000ED01A4B98420BD0194B984208D0194B37
:10471000984205D0184B984202D0184B984203D1CA
:1047200022F44072CB681A4322F080034C6943EABA
:10473000040202608B68C3620B688362054B984277
:1047400002D0084B984201D10B69036301234361F6
:1047500010BD0000002C0140000400400008004093
:10476000000C004000340140004C0140005001406A
:104770000054014000180040001C00400020004090
:1047800030B501F01F05012404FA05F3046A9C43C7
:104790000462046A01F01F0502FA05F52C43046265
:1047A00030BD000030B5056A25F001050562026ADA
:1047B0004368846924F0700424F003040D682C43DA
:1047C00022F002028D682A43104DA84200D103E076
:1047D0000F4DA84206D100BF22F00802CD682A433F
:1047E00022F00402094DA84202D0094DA84207D187
:1047F00023F4807323F400734D692B438D692B439D
:10480000436084614D684563026230BD002C014005
:104810000034014030B5056A25F010050562026AD2
:104820004368846924F4E04424F440740D6844EA45
:10483000052422F020028D6842EA0512124DA8429A
:1048400000D103E0114DA84207D100BF22F0800241
:10485000CD6842EA051222F040020B4DA84202D078
:104860000A4DA84209D123F4806323F400634D6903
:1048700043EA85038D6943EA8503436084614D689B
:104880008563026230BD0000002C0140003401400D
:1048900030B5056A25F480750562026A4368C4690B
:1048A00024F0700424F003040D682C4322F40072F9
:1048B0008D6842EA0522124DA84200D103E0114D55
:1048C000A84207D100BF22F40062CD6842EA052267
:1048D00022F480620A4DA84202D00A4DA84209D1B2
:1048E00023F4805323F400534D6943EA05138D6983
:1048F00043EA05134360C4614D68C563026230BD7D
:10490000002C01400034014030B5056A25F4805583
:104910000562036A4468C26922F4E04222F44072EC
:104920000D6842EA052223F400538D6843EA0533FB
:10493000084DA84202D0084DA84204D124F4804476
:104940004D6944EA85144460C2614D6805640362A0
:1049500030BD0000002C0140003401400EB50020A5
:1049600000900190029000BF4B48006820F00100C9
:10497000494908600920009001200190042002901C
:1049800069464648FCF7AAFB08B1FBF7E7FE424838
:10499000006840F00100404908604048FCF764FDB1
:1049A00000BF3E480068006800F002000228F8D10D
:1049B0003A48FCF743FC3A4908606FF00200374977
:1049C000096808603448006820F001003249086036
:1049D00002200090012001900420029069462F4897
:1049E000FCF77CFB08B1FBF7B9FE2B48006840F0F0
:1049F0000100294908602948FCF736FD00BF274817
:104A00000068006800F002000228F8D12348FCF793
:104A100015FC234948606FF00200204909680860CE
:104A20001D48006820F001001B490860012000902B
:104A300001900420029069461848FCF74FFB08B12A
:104A4000FBF78CFE1448006840F001001249086032
:104A50001248FCF709FD00BF10480068006800F02C
:104A600002000228F8D10D48FCF7E8FB0C498860E9
:104A70006FF002000949096808600948FCF7D4F999
:104A8000084880ED000A0648001DFCF725FA044698
:104A9000642001F0D3FB67E708240140046500208F
:104AA0007C65002010000020002600BF00250026A5
:104AB00001214FF09040FDF7C9F908B945F0010513
:104AC0004FF400511C48FDF7C1F908B945F0020543
:104AD000B5B11A4800884FF6FF71884204DA1748CA
:104AE0000088401C1549088014480088642819D1A2
:104AF000012C01D1072615E0022C13D1092611E063
:104B00000E48008805280ADD0C480088642806DA6B
:104B1000012C01D1062602E0022C00D1082600203B
:104B2000064908802C4616B13046FFF765FB0A207F
:104B300001F084FBBAE70000000800480C000020E8
:104B400008B5002400BF00BF00226946074800687E
:104B500001F0FCFD0446012C03D19DF80000FFF795
:104B600075FB642001F06AFBEEE7000008000020FE
:104B700090F8201001F0400199B10168496921F4D1
:104B80008051426A114302685161416AB1F5805F08
:104B900007D10168496921F4C041826A1143026862
:104BA0005161704770B504462168096921F440518C
:104BB000E2681143226811612269A16811436269A8
:104BC00041EA02052168C96841F20C629143294318
:104BD0002268D1602168496921F44071A2691143BA
:104BE000226851612168496921F40061E269114339
:104BF00022685161E169B1F5006F7DD1AF4A21684A
:104C0000914255D1FDF770FD00EBC00101EB0011A1
:104C100062685200B1FBF2F16422B1FBF2F10A01C9
:104C200000EBC00101EB001163685B00B1FBF3F125
:104C300000EBC00303EB001366687600B3FBF6F3EA
:104C40006426B3FBF6F303EBC30606EB0313A1EBF9
:104C50008301322303EBC1016423B1FBF3F101F0C3
:104C6000F80102EB410200EBC00101EB00116368A7
:104C70005B00B1FBF3F100EBC00303EB00136668CC
:104C80007600B3FBF6F36426B3FBF6F303EBC3063F
:104C900006EB0313A1EB8301322303EBC101642371
:104CA000B1FBF3F101F0070111442268916004E1C6
:104CB000FDF70AFD00EBC00101EB00116268520034
:104CC000B1FBF2F16422B1FBF2F10A0100EBC00189
:104CD00001EB001163685B00B1FBF3F100EBC00373
:104CE00003EB001366687600B3FBF6F36426B3FBB0
:104CF000F6F303EBC30600E032E006EB0313A1EB8F
:104D00008301322303EBC1016423B1FBF3F101F012
:104D1000F80102EB410200EBC00101EB00116368F6
:104D20005B00B1FBF3F100EBC00303EB001366681B
:104D30007600B3FBF6F36426B3FBF6F303EBC3068E
:104D400006EB0313A1EB8301322303EBC1016423C0
:104D5000B1FBF3F101F00701114422689160ACE06E
:104D6000564A2168914254D1FDF7BEFC00EBC001C8
:104D700001EB001162689200B1FBF2F100EBC0029E
:104D800002EB001263689B00B2FBF3F26423B2FBF8
:104D9000F3F202EBC20303EB0212A1EB8201322217
:104DA00002EB01116422B1FBF2F101F0F00100EB22
:104DB000C00202EB001263689B00B2FBF3F26423B3
:104DC000B2FBF3F201EB021200EBC00101EB0011A8
:104DD00063689B00B1FBF3F100EBC00303EB00132E
:104DE0006668B600B3FBF6F36426B3FBF6F303EB99
:104DF000C30606EB0313A1EB8301322303EB01117E
:104E00006423B1FBF3F101F00F01114422689160BA
:104E100053E0FDF759FC00EBC00101EB00116268A3
:104E20009200B1FBF2F100EBC00202EB00126368EA
:104E30009B00B2FBF3F26423B2FBF3F202EBC2037A
:104E400003EB0212A1EB8201322202EB0111642278
:104E5000B1FBF2F101F0F00200EBC00101EB001137
:104E600063689B00B1FBF3F16423B1FBF3F102EB48
:104E7000011200EBC00101EB001163689B00B1FB64
:104E8000F3F100EBC00303EB00136668B600B3FB5D
:104E9000F6F36426B3FBF6F303EBC30606EB03134A
:104EA000A1EB8301322303EB01116423B1FBF3F186
:104EB00001F00F0111442268916070BD003801407B
:104EC0002DE9F04104460D4617469846069E21E01E
:104ED000701CF8B12EB1FCF7C7FFA0EB0800B04280
:104EE00018D92068C06820F4D0702168C860206894
:104EF000406920F0010021684861202084F84500C5
:104F000084F8460000BF002084F8440000BF03205E
:104F1000BDE8F081206800682840A84201D1012046
:104F200000E00020B842D3D00020F1E700BFFEE748
:104F300010B500F03DF800F00DF8012251020448D0
:104F4000FCF78CFF012211020148FCF787FF10BD1E
:104F50000004004800B585B014216846FBF77DF9D0
:104F60004FF48070009011200190002002900220E8
:104F7000039069460248FCF785FE05B000BD0000BD
:104F80000004004800B585B014216846FBF765F9B8
:104F90004FF40070009000200190029002200390D6
:104FA00069460248FCF76EFE05B000BD00040048EB
:104FB00000B585B014216846FBF74FF94FF4007037
:104FC0000090112001900020029002200390694679
:104FD0000248FCF757FE05B000BD00000004004881
:104FE000014A024900F02FB8E1500008C0640020D7
:104FF00002480068C0F30220704700000CED00E09A
:1050000010B5002804DB4A07130E054A135406E0C6
:105010004A07140E034A00F00F031B1FD45410BD9F
:1050200000E400E018ED00E002E008C8121F08C12B
:10503000002AFAD170477047002001E001C1121F19
:10504000002AFBD170472DE9F04116460F46044671
:10505000002503E03946B047641C6D1C2078002809
:10506000F8D12846BDE8F0810146642201FB02F038
:1050700000E0401E0028FCD17047014601E04A1EB6
:10508000D1B20029FBD170472DE9F05F06460F46EB
:1050900090469946404600F031F88246BAF1000F3A
:1050A00001D1BDE8F09F002415E01AF804B00025F6
:1050B0000DE00120A84000EA0B0030B17A19D1B20E
:1050C0003219D0B24A46FEF7E9FC681CC5B2072D7A
:1050D000EFDB601CC4B2052CE7DB00BFE1E700009A
:1050E00013B50C464FF47A73012269460248FEF765
:1050F0008CFA00981CBD00006C6700200146202936
:1051000001DB7E2901DD00207047A1F1200000EBCA
:105110008000014A1044F7E7646F00087CB5FCF793
:10512000B5FEFBF71DFCFBF74FFCFBF7C5FDFBF7DE
:105130000DFEFBF72DFEFBF7A7FAFBF7D7FC00F0FF
:1051400015FEFFF7F5FE6E212F4881854621C185AA
:1051500088215020FEF793FEFEF7DCFD2B48FBF77D
:105160002BFF08B1FBF7FAFA2948002301220A2194
:10517000009028A001F02CFE044654B101F0DCFBA5
:105180000546002003462A4601210090204601F0F2
:105190005BFE00220121132001F064F92049086020
:1051A000002201210A2001F05DF91E49086000205B
:1051B000012103468022CDE900101BA11D4801F00A
:1051C00077FB0020012103468022CDE900101AA1BF
:1051D0001C4801F06DFB0020012103468022CDE92F
:1051E000001019A11C4801F063FB002001210346B7
:1051F0008022CDE9001019A11C4801F059FB01F0F3
:105200007FF800207CBD0000949000200465002001
:10521000D96000084175746F72656C6F616400003D
:1052200004000020080000205374617274546173FC
:105230006B000000D14200084B65794F6E4F6666E7
:1052400000000000A94A00085461736B41444346C2
:10525000756E6374696F6E005D4900085461736B0D
:1052600052474246756E6374696F6E00414B000889
:105270002DE9F04105460E46264807682648006895
:10528000001D00F00FFF50B92348006890F82C1063
:105290000120884021490968814320480160681C39
:1052A000D8B9D6B11E4948681B49096888601A49AF
:1052B00082680968CA6018490968091D82685160D6
:1052C00015490968091D8160154A134909684A6131
:1052D00011460968491C11601AE07C190E480068E3
:1052E0004460BC4207D20C480168091D0D480068A3
:1052F00000F008FF0CE008480168091D0A48006832
:1053000000F000FF09480068844201D207480460A9
:10531000BDE8F081606400204C64002064640020DB
:105320005868002054640020506400207C640020F1
:1053300010B5044600F000FF2F480068401C2E49BD
:1053400008602E48006840B92C4804600846006890
:1053500001280DD100F0D6F90AE02948006838B9D3
:1053600026480068C06AE16A884201D82348046080
:1053700024480068401C2349086094F82C10012040
:1053800088402149096808431F490860E16A01EB28
:1053900081011E4A02EB81014868A0608268E260D8
:1053A000211D826851608160E16A01EB8101174A29
:1053B00002EB81026261E16A01EB8101134A52F85A
:1053C0002110491CE26A02EB8202104B43F82210C2
:1053D00000F0C4FE0A48006868B108480068C06A66
:1053E000E16A884207D24FF0805009490860BFF354
:1053F0004F8FBFF36F8F10BD5C6400204C640020A2
:10540000686400207864002064640020B86700208D
:1054100004ED00E010B500F08FFE0C48006890B974
:105420000B4800F05FFE0B4800F05CFE08480A499C
:10543000086008480949086000220C210A2001F090
:1054400011F80249086000F089FE10BD9464002044
:105450006C680020806800208C640020906400202C
:1054600010B516E000F068FE0C48C068C468201D46
:1054700000F018FE0A480068401E09490860094803
:105480000068401E0749086000F068FE204600F0F2
:105490005FF8044800680028E4D110BD446800208B
:1054A0005C6400205864002070B504460D46206CF2
:1054B00070B1216CE0680144E160D4E902108842D7
:1054C00001D32168E1602846226CE168FAF7ACFE5E
:1054D00070BD2DE9F04104460F4615464FF0000817
:1054E000A66B206C48B9206800282CD1A06801F078
:1054F000E7FA80460020A06025E07DB93946226C9D
:105500006068FAF791FE216C606808446060D4E935
:105510000101884217D32068606014E03946226C8C
:10552000E068FAF781FE216CE068411AE1602168C9
:10553000E068884203D2216CA068411AE160022D24
:1055400001D106B1761E701CA0634046BDE8F08113
:1055500010B50446206B00F011FE204600F00EFE50
:1055600010BD00000146084A126812680AB90122FB
:1055700000E000220A600A6822B9034A1268D26871
:10558000106800E0002070478C64002030B54FF4B4
:105590002053154800F007042CB1C01D20F007006F
:1055A000114C041B1B1B0246104C226000240F4DA3
:1055B0006C60D018083820F007000D4C20600024E3
:1055C0000B4D2D686C600A4D2D682C601146441AF5
:1055D0004C60074C24680C60064D4C682C60064DEE
:1055E0004C682C6030BD000094680020A06400204E
:1055F000A8640020B0640020AC64002000BFFFF766
:105600002FFF064800680128F9D94FF0805004495F
:105610000860BFF34F8FBFF36F8FF0E7B8670020CC
:1056200004ED00E02DE9F04106460D461746984688
:10563000069C0DB9246000E02760E6632564012123
:10564000204600F035FF0020A064BDE8F0812DE980
:10565000FF5F80460E469146DDE90E7A109CA9F167
:105660000100216B01EB800B2BF0070B7EB10025B5
:1056700007E0715D04F134004155705D00B902E04E
:105680006D1C102DF5D300BF002143200155042FC0
:1056900000D30327E7626764201D00F030FD04F1AA
:1056A000180000F02CFD2461C7F10400A0616462C1
:1056B00041465846039A00F00FFB2060BAF1000FF4
:1056C00001D0CAF80040BDE8FF9F2DE9F04705462C
:1056D0000E4617469846DDE90894FFF79BFE2560C5
:1056E000A661C4F81C80C4F82090201D00F007FDBE
:1056F0002FB194F8240040F0040084F82400BDE8A1
:10570000F087000010B5002407E004EB84010F4A85
:1057100002EB810000F0E6FC641C042CF5D30C487D
:1057200000F0E0FC0B4800F0DDFC0B4800F0DAFC78
:105730000A4800F0D7FC0A4800F0D4FC04480949A4
:10574000086004480849086010BD0000B8670020E0
:10575000086800201C680020306800204468002091
:1057600058680020506400205464002010B50146A1
:10577000164800E0006803688B42FBD3024643688A
:1057800013448B4204D143684C6823444360014670
:105790000A464B6813440468A34211D10C4C0368B9
:1057A0002468A34208D04B680468646823444B60B3
:1057B00003681B680B6005E0054B1B680B6001E08C
:1057C00003680B60884200D0016010BDA064002017
:1057D000A86400202DE9F04104460D4616461F46F8
:1057E0004FF0000865602461B5420CD8F01BA16938
:1057F000884202D34FF0010811E0211D09480068DA
:1058000000F080FC0BE0BE4204D2BD4202D34FF058
:10581000010804E0211D0448006800F073FC4046C4
:10582000BDE8F081906400208C64002070B50546CE
:1058300000F082FCA86B08B9012400E0002400F00D
:105840008DFC204670BD70B5054600F075FCA86B58
:10585000E96B884201D1012400E0002400F07EFCC5
:10586000204670BDF1B50098846C0026A06BE16BFA
:10587000884221D294F94550002269462046FFF71C
:1058800028FE0646681C60B9606A08B9012000E07D
:10589000002080B904F1240001F068F958B1012614
:1058A00009E000F013FC0746BD4203D2681C40B279
:1058B00084F8450000BF00BF3046F8BD70B505460E
:1058C0000E460E480068C068C468201D00F0EAFB60
:1058D00094F8240000F0040028B1324629462046FE
:1058E00000F0C4F805E094F8240000F0FE0084F80D
:1058F00024002046216A884770BD00008C64002087
:105900007FB56EE0019800286BDB039C606908B9E5
:10591000012000E0002010B9201D00F0C3FB684604
:1059200000F0D0F8054601980A2858D2DFE800F0C8
:105930005705072E364706082F3700BF00BF00BFA8
:1059400094F8240040F0010084F824000298A26931
:10595000811803462A462046FFF73CFFA8B194F879
:10596000240000F0040038B10298A26981182A4688
:10597000204600F07BF805E094F8240000F0FE00DB
:1059800084F824002046216A884729E000BF94F863
:10599000240000F0FE0084F8240021E000BF94F809
:1059A000240040F0010084F824000298A061A0695E
:1059B00041192B462A462046FFF70CFF10E094F8C9
:1059C000240000F0020018B9204600F0D7FB05E0E3
:1059D00094F8240000F0FE0084F8240000E000BFEA
:1059E00000BF002201A90348006800F0AFFE0028B4
:1059F00088D17FBD94640020F8B505460C4600F0C0
:105A0000BBFC684600F05EF80646009820BB44B92F
:105A1000B54206D801F02EF931462846FFF74EFF71
:105A20001CE03CB10E480068006808B9012000E0A5
:105A300000200446A91B22460A48006800F0D8FB53
:105A400001F018F950B94FF0805007490860BFF3D2
:105A50004F8FBFF36F8F01E001F00CF9F8BD00002C
:105A6000906400209464002004ED00E070B50446CA
:105A70000D46164604E0A06905442046216A884781
:105A8000A06941192B4632462046FFF7A3FE0028A5
:105A9000F1D170BD09480068006808B9012000E034
:105AA000002020B14FF0FF300549086005E00348B1
:105AB0000068C068006802490860704750640020B0
:105AC0007C64002070B5044600F036FF05460748A8
:105AD0000068854204D200F00BF80120206001E04C
:105AE0000020206001480560284670BD9C640020AD
:105AF00070B508E00D480068C06804684FF0FF31D9
:105B00002046FFF7DBFE09480068006808B901205D
:105B100000E000200028EDD0044805680448006833
:105B2000024908600248056070BD00008C640020D6
:105B30009064002000BF502080F31188BFF34F8F86
:105B4000BFF36F8F00BF00BFFEE708B500BF684618
:105B5000FFF708FD044620460099FFF74DFFFFF7C9
:105B6000CFFEF4E770B5044600F0E6FA94F945502C
:105B700019E0A06C30B12046FFF774FE88B100F048
:105B800083FB0EE0606A08B9012000E0002038B90C
:105B900004F1240000F0EAFF18B100F075FB00E00A
:105BA00003E0681E45B2002DE3DC00BFFF2084F84F
:105BB000450000F0D3FA00F0BFFA94F9445010E029
:105BC000206908B9012000E0002048B904F1100064
:105BD00000F0CCFF08B100F057FB681E45B200E0B2
:105BE00001E0002DECDC00BFFF2084F8440000F051
:105BF000B5FA70BD2DE9F04705464FF0000900F0F9
:105C0000BBFB3048006808B9FFF7C0FC75B105F070
:105C10000700C0F11008C8F1FF30A84201D20120EE
:105C200000E0002008B9454400E00025012000EB19
:105C3000E570002841D0002D3FD023480068854200
:105C40003BD8224E3046046801E02646246860684E
:105C5000A84202D220680028F7D11A48006884427E
:105C60002BD0306800F10809206830606068401B64
:105C7000102807D967196068401B7860656038464E
:105C8000FFF774FD104960680968081A0E4908603A
:105C9000084600680E490968884203D20A4800682D
:105CA0000B490860606840F00040606000202060A0
:105CB00008480068401C0749086000F0DBFF4846C0
:105CC000BDE8F087A8640020AC640020A064002038
:105CD000B0640020B4640020001F4FF080730360A4
:105CE000001F21F001030360001F054B03601438FF
:105CF0000260001F6FF0020303602038704700004D
:105D0000355B000870B505462E46002406E00121EB
:105D1000A14001EA060000F005F8641C182CF6DB2F
:105D200070BD000010B504466CB1012280210E4800
:105D3000FCF794F80620FFF7A0F9002280210A481A
:105D4000FCF78CF80FE0012280210748FCF786F869
:105D50000220FFF792F9002280210348FCF77EF829
:105D60000320FFF78AF910BD0004004810B584A095
:105D7000FFF736F900F016F900224FF4006184486D
:105D8000FCF76CF86420FFF76FF90122D10280481C
:105D9000FCF764F842F21070FFF766F91120FDF786
:105DA0000DFF4FF47A70FFF75FF92820FDF706FF2B
:105DB000B120FDF703FF0520FDF7EAFE3A20FDF7CD
:105DC000E7FE3A20FDF7E4FEB220FDF7F7FE0520DE
:105DD000FDF7DEFE3A20FDF7DBFE3A20FDF7D8FEA8
:105DE000B320FDF7EBFE0520FDF7D2FE3A20FDF7CC
:105DF000CFFE3A20FDF7CCFE0520FDF7C9FE3A2084
:105E0000FDF7C6FE3A20FDF7C3FEB420FDF7D6FE2F
:105E10000320FDF7BDFEC020FDF7D0FE0E20FDF7EC
:105E2000B7FE0E20FDF7B4FE0420FDF7B1FEC12041
:105E3000FDF7C4FEC020FDF7ABFEC220FDF7BEFE9D
:105E40000D20FDF7A5FE0020FDF7A2FEC320FDF703
:105E5000B5FE8D20FDF79CFE2A20FDF799FEC4209B
:105E6000FDF7ACFE8D20FDF793FEEE20FDF790FED2
:105E7000C520FDF7A3FE0E20FDF78AFE3620FDF7B4
:105E80009DFE0820FDF784FEE020FDF797FE102020
:105E9000FDF77EFE0E20FDF77BFE0220FDF778FE6B
:105EA0000320FDF775FE0E20FDF772FE0720FDF7BB
:105EB0006FFE0220FDF76CFE0720FDF769FE0A2049
:105EC000FDF766FE1220FDF763FE2720FDF760FE5A
:105ED0003720FDF75DFE0020FDF75AFE0D20FDF78F
:105EE00057FE0E20FDF754FE1020FDF751FEE12075
:105EF000FDF764FE1020FDF74BFE0E20FDF748FE77
:105F00000320FDF745FE0320FDF742FE0F20FDF7BD
:105F10003FFE0620FDF73CFE0220FDF739FE08207B
:105F2000FDF736FE0A20FDF733FE1320FDF730FEA5
:105F30002620FDF72DFE3620FDF72AFE0020FDF776
:105F400027FE0D20FDF724FE0E20FDF721FE102078
:105F5000FDF71EFE3A20FDF731FE0520FDF718FE85
:105F600000F09BF81F20FDF7B5FD4FF4784309A220
:105F700014210A20FDF7F6FD08A0FFF731F810BD47
:105F8000646973706C617920696E69742000000027
:105F90000004004868656C6C6F0000004F4B0D0AF0
:105FA0000000000000B587B000BF2948406B40F0FA
:105FB0000800274948630846406B00F0080001903C
:105FC00000BF00BF0815029001200390002004903C
:105FD0000220059002A91F48FBF754FE4FF4006011
:105FE000029001200390002004900220059002A955
:105FF0001848FBF747FE4FF48050029001200390B1
:10600000002004900220059002A91248FBF73AFEF6
:106010004FF4804002900120039000200490022061
:10602000059002A90B48FBF72DFE01221103094838
:10603000FBF714FF012291030648FBF70FFF012233
:10604000D1020448FBF70AFFFDF764FD07B000BD6D
:1060500000100240000400482DE9F04104460D46BE
:1060600016461F462A20FDF7A9FD04F1180188B243
:10607000FDF797FD05F1180188B2FDF792FD2B2081
:10608000FDF79CFD3046FDF78CFD3846FDF789FD98
:106090002C20FDF793FDBDE8F08110B52920FDF718
:1060A0008DFD10BD01460A69D1E901309860D1E942
:1060B000010358605068884201D188685060002010
:1060C00008611068401E1060106870470148006841
:1060D000704700005C64002010B504460220FEF703
:1060E00099F810BD00F1080141604FF0FF31816067
:1060F00000F10801C16001610021016070470021C9
:106100000161704710B502460B685C1C0CB9106940
:1061100007E002F1080000E04068446824689C42FF
:10612000FAD944684C604C68A160886041600A619B
:106130001468641C146010BD00BF502080F31188E7
:10614000BFF34F8FBFF36F8F00BF03480068401C41
:106150000149086070470000BC64002006480068E0
:10616000401E054908600846006820B9002080F3F9
:10617000118800BF00BF7047BC64002070B50646A0
:106180003546E6B1083D2C466068C00FB8B12068BE
:10619000A8B9606820F00040606000F0EDF80849A0
:1061A000606809680844064908602046FFF7DEFA7F
:1061B00004480068401C0349086000F05BFD70BDA6
:1061C000AC640020B864002000204FF0E02108619A
:1061D0008861064800684FF47A71B0FBF1F0401E08
:1061E0004FF0E0214861072008617047000000205F
:1061F0002DE9F04105460E4617462C46FFF79CFF59
:1062000094F94400401C10B9002084F8440094F92B
:106210004500401C10B9002084F84500FFF79EFFA0
:10622000A06B28B93A46314604F1240000F042F848
:106230002046FFF797FCBDE8F081000070B50446EA
:10624000002544B100F098F800212046FFF710F82F
:1062500000F010FD05463DB94FF08050034908603D
:10626000BFF34F8FBFF36F8F70BD000004ED00E0F0
:1062700003490968016003490968416070470000EB
:1062800074640020606400200120014908607047A8
:106290007064002070B505460C4605480168183149
:1062A0002846FFF72FFF01212046FEF7E1FF70BDD2
:1062B0004C64002070B504460E46154660680F49D0
:1062C0000968C8610D49826809680A620B49096852
:1062D000183182685160094909681831816007499D
:1062E00009688C622168491C21600DB14FF0FF36AE
:1062F00029463046FEF7BCFF70BD00004C6400200C
:106300001CB5154800210B464FF40072CDE9001072
:1063100012A1144800F0CCFA0446012C02D100F07E
:1063200073FD0446012C14D100BF502080F3118866
:10633000BFF34F8FBFF36F8F00BF4FF0FF300A499D
:10634000086001200949086000200949086000F040
:106350004BF8084800681CBD8064002049444C4547
:1063600000000000FD5500087C64002068640020E7
:10637000606400208464002002480068401C0149D9
:1063800008607047886400201248006818B1012036
:10639000114908601DE000200F4908600F4800689F
:1063A000B0FA80F0C0F11F0101EB81020C4B03EB4E
:1063B000820042685268426000F1080243689342DA
:1063C00002D14268526842604268D268054B1A6046
:1063D00000BF70478864002070640020646400205F
:1063E000B86700204C64002010B50E48006840F4E7
:1063F00070000C4908600846006840F07040086072
:10640000FFF7E2FE002008490860F9F7BFFE0748E1
:10641000006840F0404005490860F9F7A3FE0020FD
:1064200010BD000020ED00E0BC64002034EF00E06F
:1064300010B500BF502080F31188BFF34F8FBFF31A
:106440006F8F00BF00F07EFA18B14FF08050044902
:10645000086000BF002080F3118800BF10BD00005D
:1064600004ED00E02DE9F84304460E4617460025EA
:10647000DCB1681EB0FBF4F0B04216D304FB06F0AA
:1064800010F14D0F11D804FB06F909F14C00FFF78C
:10649000B1FB05464DB1A84608F14C083B464246C3
:1064A000314620460095FFF7BDF82846BDE8F88341
:1064B0002DE9F04105460E4601272C46002C41D01F
:1064C000E06B00283ED0B91EE06BB1FBF0F0216C10
:1064D000884237D3FFF730FED4E90F12206801FB62
:1064E0000200A0600020A06320686060E06B401E96
:1064F000226C216800FB0211E160FF2084F8440057
:1065000084F845009EB9206908B9012000E0002008
:10651000A8B904F1100000F029FB80B14FF08050C1
:106520000A490860BFF34F8FBFF36F8F07E004F194
:106530001000FFF7D7FD04F12400FFF7D3FDFFF7AC
:106540000DFE00E000273846BDE8F08104ED00E0D4
:106550002DE9FF4782B0074688461D464FF00009E7
:106560003C4600BFFFF7E8FDA06BE16B884201D31A
:10657000022D3ED1D4F838A02A4641462046FEF7E7
:10658000A8FF0646A06C88B1022D02D1BAF1000F17
:1065900029D12046FFF766F928B34FF080503D49D6
:1065A0000860BFF34F8FBFF36F8F1CE0606A08B9BC
:1065B000012000E0002068B904F1240000F0D6FAC0
:1065C00088B14FF0805033490860BFF34F8FBFF35D
:1065D0006F8F08E03EB14FF080502E490860BFF346
:1065E0004F8FBFF36F8FFFF7B9FD012006B0BDE8F5
:1065F000F087049818B9FFF7B1FD0020F6E7B9F16C
:10660000000F04D16846FFF733FE4FF00109FFF792
:10661000A5FDFFF7B1FEFFF78FFD94F94400401C84
:1066200010B9002084F8440094F94500401C10B9CA
:10663000002084F84500FFF791FD04A9684600F0AA
:1066400007F9F8B92046FFF7FEF8A8B104F11000E9
:106650000499FFF71FFE2046FFF784FA00F00AFBBB
:1066600000287FF47FAF4FF080500A490860BFF3E5
:106670004F8FBFF36F8F75E72046FFF773FA00F077
:10668000F9FA6FE72046FFF76DFA00F0F3FA002001
:10669000ACE7000004ED00E02DE9FF4F81B00646B5
:1066A00015461F46344600BF5021EFF3118081F399
:1066B0001188BFF34F8FBFF36F8F00BF8146A06B70
:1066C000E16B884201D3022F36D194F945A0A06B2B
:1066D00000903A4620460299FEF7FBFE0AF10100BF
:1066E000E0B9A06C58B1022F01D1009808BB204638
:1066F000FFF7B8F8E8B1E5B10120286019E0606A59
:1067000008B9012000E0002098B904F1240000F04D
:106710002DFA70B16DB1012028600AE0FFF7D6FCB8
:106720008346DA4504D20AF1010040B284F84500FC
:1067300000BF4FF0010801E04FF0000800BF89F3EF
:10674000118800BF404605B0BDE8F08F2DE9F74144
:1067500083B005460F464FF000082C4600BFFFF7F8
:10676000EBFCA66BF6B139462046FEF79DFE701E87
:10677000A063206908B9012000E0002060B904F19D
:10678000100000F0F3F938B14FF080502F49086045
:10679000BFF34F8FBFF36F8FFFF7E0FC012006B010
:1067A000BDE8F081059818B9FFF7D8FC0020F6E79E
:1067B000B8F1000F04D101A8FFF75AFD4FF001080E
:1067C000FFF7CCFCFFF7D8FDFFF7B6FC94F94400C7
:1067D000401C10B9002084F8440094F94500401C86
:1067E00010B9002084F84500FFF7B8FC05A901A8FE
:1067F00000F02EF8F0B92046FFF718F8A0B104F128
:1068000024000599FFF746FD2046FFF7ABF900F09D
:1068100031FA0028A3D14FF080500C490860BFF333
:106820004F8FBFF36F8F9AE72046FFF79BF900F079
:1068300021FA94E72046FFF795F900F01BFA20466D
:10684000FEF7F4FF00288AD00020A8E704ED00E05E
:1068500070B506460C46FFF76FFC13480268706877
:10686000131A2068401C08B9002519E00F49306848
:106870000968884206D07068904203D8012500203C
:1068800020600DE02068984207D92068C01A206077
:106890003046FFF7EDFC002502E0002020600125D6
:1068A000FFF75CFC284670BD606400207464002023
:1068B0002DE9FF4F85B0804689461746DDE912ABCA
:1068C000B800FFF797F9064676B15420FFF792F922
:1068D00004462CB154212046F9F7BFFC266304E09E
:1068E0003046FFF74BFC00E000247CB10020CDE9EE
:1068F00000ABCDE902403A4649464046089BFEF7C8
:10690000A6FE2046FEF714FD012501E04FF0FF35FD
:10691000284609B0BDE8F08F0549096809B901208A
:1069200005E00449096809B9022000E00020704729
:1069300068640020886400200149086870470000EE
:10694000606400202DE9F0410027524800680028CB
:106950007ED151480068451C4F4805608DB94F48AD
:10696000D0F800804E4800684C4908604C48C0F898
:1069700000804C480068401C4A490860FFF78AF8CC
:1069800000BF49480068854276D300BF434800688D
:10699000006808B9012000E0002020B14FF0FF306E
:1069A0004149086067E03D480068C068C46866689F
:1069B000B54202D23C4806605DE06069D4E902124B
:1069C0008A60D4E902214A60211D42688A4201D1CD
:1069D000E1684160002262610168491E0160A06AAD
:1069E00098B1A06AD4E907128A60D4E907214A6005
:1069F00004F1180142688A4201D1216A41600022F3
:106A0000A2620168491E016000BF94F82C100120A9
:106A1000884026490968084324490860E16A01EB77
:106A20008101234A02EB81014868A0608268E2602C
:106A3000211D826851608160E16A01EB81011C4A7D
:106A400002EB81026261E16A01EB8101184A00E018
:106A500017E052F82110491CE26A02EB8202144B43
:106A600043F822101349E06A0968C96A88428DD93F
:106A700001278BE700E000BF0F48006800B1012745
:106A800004E00E480068401C0C4908603846BDE828
:106A9000F0810000886400206064002050640020C1
:106AA00054640020746400207C640020646400202E
:106AB000B86700204C640020706400206C640020E3
:106AC00070B505462C460026002D48D0A06C401E0F
:106AD000A064616CE06A884241D0A06C00283ED17D
:106AE000201DFFF7DFFA40B994F82C1001208840F0
:106AF0001C49096881431B480160606CE062E06AE0
:106B0000C0F10400A06194F82C10012088401549C0
:106B10000968084313490860E16A01EB8101124AE0
:106B200002EB81014868A0608268E260211D8268F2
:106B300051608160E16A01EB81010B4A02EB810245
:106B40006261E16A01EB8101074A52F82110491C98
:106B5000E26A02EB8202044B43F82210012630461F
:106B600070BD000064640020B867002070B5034663
:106B7000D868C168886AD1E90745A560D1E907549A
:106B8000656001F118044568A54201D10C6A4460B2
:106B900000258D620468641E046030480068002887
:106BA0003DD14869D1E90245A560D1E9025465604B
:106BB0000C1D4568A54201D1CC68446000254D619B
:106BC0000468641E046091F82C400120A040244C0D
:106BD00024682043224C2060CC6A04EB8404214DBD
:106BE00005EB8404606888608568CD600C1D85684D
:106BF0006C608460CC6A04EB84041A4D05EB840558
:106C00004D61CC6A04EB8404164D55F82440641C95
:106C1000CD6A05EB8505134E46F8254010E0124C71
:106C20006068C86185680D6201F1180485686C6050
:106C300084600D4D8D622C462468641C2C6000BF5E
:106C40000A4CC86A2468E46AA04204D901220120DF
:106C5000074C206000E00022104670BD88640020D0
:106C600064640020B8670020306800204C64002075
:106C70007064002070B500240026FFF75DFA4B48D1
:106C80000068401E494908600846006800287DD118
:106C900047480068002879D05BE04648C068C4686F
:106CA000A06AD4E907128A60D4E907214A6004F196
:106CB000180142688A4201D1216A41600022A26221
:106CC0000168491E01606069D4E902128A60D4E952
:106CD00002214A60211D42688A4201D1E168416077
:106CE000002262610168491E016094F82C100120A5
:106CF00088403149096808432F490860E16A01EB7F
:106D000081012E4A02EB81014868A0608268E2603E
:106D1000211D826851608160E16A01EB8101274A8F
:106D200002EB81026261E16A01EB8101234A52F8C0
:106D30002110491CE26A02EB8202204B43F8221028
:106D40001F49E06A0968C96A884202D301201D49C7
:106D500008601848006808B9012000E000200028F9
:106D60009BD00CB1FEF796FE1748056865B100BFD1
:106D7000FFF7E8FD10B10120124908606D1E002DDB
:106D8000F6D10020104908600E4800E009E00068D4
:106D900038B1012630070D490860BFF34F8FBFF3AC
:106DA0006F8FFFF7DBF9304670BD0000886400206C
:106DB0005C6400203068002064640020B867002014
:106DC0004C640020706400206C64002004ED00E03E
:106DD0002DE9FC4705460E4617469846DDF82890F3
:106DE0002820FEF707FF044654B1002084F8240051
:106DF00043463A4631462846CDE90094FEF765FC05
:106E00002046BDE8FC8700001CB50024FEF702FB0D
:106E10000848006858B10848032100234FF48062F5
:106E2000CDE9001005A10748FFF742FD04462046C2
:106E30001CBD00009464002098640020546D7220F2
:106E4000537663004B5B00082DE9FE4305460C4674
:106E500016461F46DDF828804FF0000914480068E8
:106E600010B3009401960295062C15DAFFF754FD35
:106E7000022808D10023424669460D480068FFF702
:106E800067FB814610E000231A46694608480068FF
:106E9000FFF75EFB814607E000233A466946044857
:106EA0000068FFF7F9FB81464846BDE8FE83000015
:106EB00094640020000000000000000001020304B0
:106EC0000607080900000000010203041051FF1F1B
:106ED0001451FF1F1851FF1F4851FF1F4C51FF1F36
:106EE0000056FF1F0456FF1F0052FF1F0452FF1FD2
:106EF0004051FF1F4451FF1F0852FF1F2051FF1F29
:106F00002451FF1F2851FF1F2C51FF1F3051FF1F1D
:106F10003451FF1F082202400C220240202202406E
:106F200028220240242202401C2202402C2202403D
:106F3000102202401422024018220240FF0FFF0FCD
:106F4000FF0000000F001F00FF07FF1FFF07FF07E4
:106F50003F003F003F000000FFFFFFFFFFFFFFFF7C
:106F6000FF0FFF0F000000000000005F000000079F
:106F7000000700147F147F14242A7F2A1223130889
:106F8000646236495522500005030000001C22416E
:106F9000000041221C00082A1C2A0808083E080894
:106FA0000050300000080808080800606000002059
:106FB000100804023E5149453E00427F40004261B4
:106FC0005149462141454B311814127F1027454540
:106FD00045393C4A49493001710905033649494957
:106FE00036064949291E0036360000005636000094
:106FF000000814224114141414144122140800022D
:1070000001510906324979413E7C1211127C7F49B7
:107010004949363E414141227F4141221C7F494935
:1070200049417F090909013E4149497A7F08080819
:107030007F00417F41002040413F017F08142241F1
:107040007F404040407F020C027F7F0408107F3E5B
:107050004141413E7F090909063E4151215E7F09B8
:10706000192946464949493101017F01013F404004
:10707000403F1F2040201F3F4038403F631408140A
:107080006307087008076151494543007F4141008B
:1070900002040810200041417F0004020102044064
:1070A00040404040000102040020545454787F487E
:1070B0004444383844444420384444487F38545485
:1070C0005418087E090102081454543C7F08040433
:1070D0007800447D40002040443D007F102844005B
:1070E00000417F40007C041804787C080404783850
:1070F000444444387C14141408081414187C7C0884
:107100000404084854545420043F4440203C404068
:10711000207C1C2040201C3C4030403C442810284F
:10712000440C5050503C4464544C440008364100D8
:1071300000007F0000004136080008082A1C0800F3
:107140000000000000005F00000007000700147F3F
:10715000147F14242A7F2A122313086462364955A7
:1071600022500005030000001C2241000041221CA7
:1071700000082A1C2A0808083E08080050300000B1
:107180000808080808006060000020100804023E9B
:107190005149453E00427F400042615149462141EC
:1071A000454B311814127F1027454545393C4A4953
:1071B00049300171090503364949493606494929CB
:1071C0001E0036360000005636000000081422412A
:1071D0001414141414412214080002015109063237
:1071E0004979413E7C1211127C7F494949363E4122
:1071F0004141227F4141221C7F494949417F090980
:1072000009013E4149497A7F0808087F00417F41D2
:10721000002040413F017F081422417F4040404010
:107220007F020C027F7F0408107F3E4141413E7F78
:10723000090909063E4151215E7F0919294646493F
:1072400049493101017F01013F4040403F1F20403B
:10725000201F3F4038403F6314081463070870083C
:10726000076151494543007F414100020408102055
:107270000041417F000402010204404040404000C0
:107280000102040020545454787F48444438384460
:10729000444420384444487F3854545418087E09E4
:1072A0000102081454543C7F0804047800447D40D3
:1072B000002040443D007F1028440000417F4000F2
:1072C0007C041804787C0804047838444444387CEE
:1072D00014141408081414187C7C08040408485476
:1072E000545420043F4440203C4040207C1C20401B
:1072F000201C3C4030403C44281028440C50505046
:107300003C4464544C44000836410000007F0000B7
:10731000004136080008082A1C08A0002405A40122
:1073200021A46AEC13437AE144204820FA211B216E
:107330002D21617ACFEAE643F14429E07AC8E7419A
:1073400032AB03860192196AF4437AE3446AF2434A
:107350007AE4446AEF437AE5446AF04121DF7AE651
:107360004521BE017ACEC4E6437AF14429CC6AF6BF
:1073700044AA067AF2E7416AF6457ACEC6E6437A2F
:10738000F14429CC6AF744AA067AF2E7416AF74544
:107390007ACEC8E6437AF14429CC6AF844AA077A3F
:1073A000C7F4E6416AF8457ACECAE6437AF1442941
:1073B000CC6AF944AA077AC3C8E6416AF9457ACE8D
:1073C000D0E6437AF14429E07AC1E74132AB457A0D
:1073D000CED0E6436AFA447AC0E7436AFB4422030C
:1073E0007ACECCE6437AF14429A67AC1E7414B1222
:1073F00030AB216AEF446AF5446AF4455B7AD6E71C
:10740000436AF3447ACED1E6436AFA447ACAE74340
:107410006AFB442203027AD94121CD7AE2457ADE21
:107420004121F16AEE457AE8456ADA436AE6415D50
:107430006AED457AE745026AED436AF6415CAD06BE
:10744000706AF2455B920060027AD4E7416AF35AAF
:10745000AD0C136AEE436AEF446AF0455B921C6A16
:10746000EE436AEF415C6AF044A90149116AF144B4
:107470006AF7415CAD027192026192FF02B837B9BE
:10748000256AF413416AF9435CAD0F6AF5436AEE6D
:107490004154466AF5446AF41392236AF4455B6AE0
:1074A000F5436AEF4492176AF213416AF8435CAC01
:1074B0000D6AEE436AEF446AF4455B6AF2455B028B
:1074C00060617AC4E1437AE03A6AEC455B6AF3456D
:1074D0005B6AF4455B6AF2455B02C1D8243E9000CA
:1074E0007F666776776699FD02C0C5C9270C6AC4B6
:1074F000416AC552526AC652474702CACFD3270CC7
:107500006ACE416ACF52526AD052474702D4E0EB6A
:10751000270C6ADF416AE052526AE1524747027A19
:10752000C3D4E6437AF0446AFA437AF1446AFB43EF
:107530007AF2442A557AC0E7437AF04402A3C001A4
:1075400090F81081000C08007D0000000800000089
:1075500050000080010430770052005A00010808F2
:10756000005740000000710000080000000001000A
:10757000000000009475000800000020C4640000B2
:107580003E05000854CC0008C464002014300000FC
:107590003850000800061500D8B805000112030491
:1075A000920810120110100F71A561445103598502
:1075B000596461A45984023012646185698571C679
:1075C00069A571E661C66A0672270220084772271C
:1075D0007A68828904200982A97A688ACA8AEA04B8
:1075E00023932B04500D9B2B9B2C9B6C9B6C936CBF
:1075F0008B2B0410040B8B2B1010060B930B9B4C46
:107600002E13EB8B0A13930B3C200E8A8AEB828994
:107610008AAA8ACA61E66A07084015496428C272C4
:10762000AA8B8DFFFFF79DF77DF77CEF5BEF7B0467
:107630002029FFDCB40AAB4671A5698540C261C64A
:1076400069E66A067A677227510372077A07822809
:1076500082887227594469E682888E10058288598B
:10766000430C12A95C1008CA82A959647207A011C0
:1076700002111813647A141005930B8AEA3C200651
:10768000438B0A8B0AB42005722761A69E119612BD
:107690000ADE2006488B0B92EBA03369A62C100E55
:1076A000AA92EA40C26A278AA992EB4144A0428981
:1076B000A01029EF5CEF5CB594BDB4BDD5B5B4B5F1
:1076C000D5FF7ABC4BAB46698569A648C269E669B5
:1076D000C561A57A477A27720769A5A03004487A60
:1076E000070C12C6A02647342371E79410067A4887
:1076F00082AA82A2177A484220088992EB92EB7AFA
:10770000897E152814086C8ACA720792EB54120BF2
:1077100010300A2B72279B4C92EA9B0BBA134893AA
:107720000C219811381406EB8ACA92CA3810092322
:1077300062068AAA82AA49A050056A6993CEA0125D
:107740003B02100C5AE71AE73AEF7BFFFCABE9A0CB
:1077500027A56140100EC569A569C5720672066944
:10776000C669C69C2207AC310C1404488268D61046
:107770001EA972276A276A07728972687AA959C690
:10778000620772697AAA932C8AEB72A97288B21185
:1077900072212415F831023008930B7207930B9273
:1077A0008A410C11961AEA2021A032AAA040104466
:1077B00061C68AA98AEA496530E26A699C0FA054C9
:1077C0000CE73BEF5BDEF9DEF9E73AE7E015382836
:1077D000068448E261A570100571E67A06A83006B5
:1077E000A57A287A06AC11BC138248021540101500
:1077F00061E649645A273923394349E53143314326
:1078000041A539640E28086449A562687AAA601502
:107810004A1207A0117E1A929C137206A016EA64FF
:1078200011BA177228F4211632AA22180BEA8AA973
:1078300082A9492361E68A2E11A06006C26A489C8B
:1078400030A013E73AA016FA42263B4027A325D8DA
:10785000334902A02006A571C679E6942540177227
:1078600006401004A55944AC1A689C20102751A565
:10787000414331023143210220E231840212210EC0
:10788000140E2903314349A559E77AAA82EB7AF607
:10789000378269BE3408A98ACA69E68AEA401406B2
:1078A000AA8AC97A28361404A98AC94036286219D6
:1078B000C82005516461E6F881A01409EF9DEF7DB1
:1078C000EF3BE6FA401006D9DEFAEF5CA01404C9DB
:1078D000B366E015401C0B598471C671C67A0679EF
:1078E000E6D003176479481771E6EC1994301172E9
:1078F000487288390228A1418441C541E529239C69
:107900001264082C186441C639644A2739A54A060E
:1079100051E6624862276A686206728942031184EE
:1079200032C9A0152A210225361292AE400582489E
:1079300071E7A0198010040359C5CE2EEA20032058
:10794000056A48A450A017F79D40163BDE14041AA0
:10795000E75BE011A01011A30569846164514359EC
:107960008469C571C579E6A02004C6696508198CCB
:10797000140D2661A561C6622749A528A139D0202A
:107980001F49E64206292339C54207316439C641F9
:10799000C649E7524831644A4739A55A6852070236
:1079A00011A817477ABC2DE80335CA154A1196214C
:1079B0000C41AA39021D660419D024044103594020
:1079C000200789412328C262A032FEA024041BEFB5
:1079D0005BE4198828089CFFFCA3A8AB45701D0038
:1079E000051264A012E59E1EC5700415401429718D
:1079F000C672266A0661E659E638E2416531033906
:107A00006441855A4841E6316431645248398541C0
:107A1000E641C64A07524844140A65526852486211
:107A2000A95A886027A5524215DE500582A969C669
:107A300094554011AA11A0137A271E1DA6041C04F8
:107A4000828841C0031D0E0442CAA015E011A01394
:107A5000EF7D981D02051009E75BEF7CF7BDFFDCA9
:107A6000A01E2500051C06A55123514390052EC5D7
:107A700022031D700420048579E7A0100B620651D3
:107A800084392328A128C2A0300C6552485A695273
:107A9000283144292396100C8539A5318552884A0E
:107AA0004839A5961227A21806EA39844A068C1F7F
:107AB000C672840424078AA971E68AC93245E05552
:107AC000EA21A011C031A01C040361E6AE04100439
:107AD000A93903A07A28802E7C04051102329DA0CA
:107AE0003C0A88AB25698469855123220315421D10
:107AF00034062C04445924FC0424056A0659E5D8AC
:107B0000240720E22923188138240D5A6939A64A0E
:107B10000741E742075268E4100B41E62923736CE2
:107B2000396541A6BC1012686B0A734B526849E66E
:107B300072896A277A697A48A032899E15CE51A047
:107B400040068982697207A0637A68A01338E3A0AF
:107B50005E2720033E7CA40510067CEF7DF7BDA0C8
:107B600012BCA0300845696469855943A022E5022A
:107B70001F5944E006100CE669E6728851C520A141
:107B800020C19A1408A52944210308202226C6CC26
:107B9000240F39A552484A4831854A4821034A48AA
:107BA000DC1C1141A6732B5A8983EE31435A686A53
:107BB000A96A681C0532898A1C04488A683E051E29
:107BC0002716032D54041C0488824890062A6976DF
:107BD00061A04C097A8930C228A262072003219A49
:107BE000110471A01B9B678015401F59440205308A
:107BF000048569C502141AE6598572486A2759E650
:107C0000498428E2188039C539C639C618A11081BF
:107C10002C1406855A894A28D22410A6734C5289FE
:107C200042075AA920E37BAD5A89FA1C0F734C73A3
:107C30006C732B41A572EA832B6227560615CA1C6A
:107C4000048A698A3E051D86062EE66E061DE80535
:107C50001E48F0051268A8110A1D20031406C672FA
:107C6000287A69403806A16207AC918041A221A41C
:107C700025E022BBA01C0D61646184514348C161B1
:107C80008469A53E061DB607140D6A07830A59C507
:107C90004143396320E22C140C68398439A520E271
:107CA00018A16B0BCA1C2C6962CA4A2752686B2C3C
:107CB0006B4C4A487B8E29237BAD6B0B5A896ACA71
:107CC0005A687B6C8C0F62A96268836C9BEE7AEABF
:107CD0006A07980715422D2A073DBA0721961D927B
:107CE00006197C1669F23247A05004077248A0209A
:107CF00004B1FFDE94197A21A0498040049B9B4780
:107D0000A0175943401C068469847A47A8081C0AB6
:107D100088830A7AC949643963B4031C07E64A07B1
:107D20005A89414C04198624040252272820056BE5
:107D30000B52899E10098C303165736D630BA61C44
:107D400019CD4A2762AA52487B8D8C0F942F6AEA7C
:107D50007B6B8BCD838C8B8C7216071D4A04164867
:107D6000E02D4A04310A21A0167A48437227A01751
:107D70007A48E043C25AA057BDF7E2A2E7A02E44DA
:107D800000051748C2481816647A476A47832B9340
:107D9000AD5A065A473963524741C652475E1D885D
:107DA00005142128E229033985734C4A28630B7393
:107DB0008E4A28840FB59539C69471738D39E78C36
:107DC00070630B3A2C14CA732B9C91944F83AD941F
:107DD0002F8C0E7B4BA44F9BCD94091964198025E1
:107DE0003411FE2D7C081D3C031D7A0821A012A62B
:107DF000A030046930A2A0140491FFDE3E02127D7F
:107E0000A01C076964594340C10205140CE66A4886
:107E10008B6C838C734B5A272C1C054752475A98FE
:107E2000031F734CEC041DAA031DCA06201E446BDD
:107E30000B4A07736D6B2C4208738E8C305ACA8CB8
:107E400050736D318584106B2C8C0FA21011840E31
:107E5000AD539490AD1283ED7B6B83AC9C0EA2115D
:107E6000961D200726C6481D3E061EE624091E68EC
:107E70009206240827722840E259A5E02D20032EFF
:107E80005A200315407D2003498010087B9306ABE0
:107E9000256123A01264A01C0E8549237ACA9C4F39
:107EA000734B7BAC49E610061C0548730B5A7805EA
:107EB0002B734C841433290228E3398562EB29445F
:107EC000630C528A29656B4D4A495AAA94715AAA81
:107ED00020E3736D736D945083EF738D94909CD1F8
:107EE000AD53C5F5A4D083CD421C076FAC909BCD9C
:107EF0007AB4083B6164883E481804124802362868
:107F00004041A022A2A0229CA0529D9C71A0339B24
:107F100026A01C2084490238A1516449449BEE628A
:107F20006862EA62EA31236ACA7B6C6AEA4A0652EC
:107F300006732B6A0717A531401DC80614368A2917
:107F400004524931862924630C4A2842077BAE52E9
:107F50004820E36B2C4A288C5062CA6B0B734CA4EC
:107F6000D18C2F83CDBD93AD12732A9C6FACB1B46D
:107F7000D18B2B401EC54A041DA8092D660A2DAEC3
:107F80000A900572286A07A02C04C2620760093DA6
:107F9000BA03A540225AA01B5902802C1C2338A1E9
:107FA00059A57AEA834C62896AEA6B0A31447B4CB0
:107FB0005A685A8849C641A4B8061DC2031A64808B
:107FC0001C0F6541C629443186318520E3528A3928
:107FD000E00614295AA94A072944526841E6528901
:107FE0004A0783CE5AA983CD6B0B7B6C942FBD734C
:107FF0009C6FA490ACF1ACB0AC706A47D611A025D0
:10800000401F61C5440AA1A04A28807393EEA03D99
:10801000A00581A01E58BA032C15596438C159A572
:10802000830B4143628862C94A2741A5838D1008AA
:108030001DDE091C06E5520639632E0321A01E84AD
:10804000C8033C10E339A63165108241E720E35AAA
:108050006962A98C071C06C6524842071C051DDE32
:10806000031F5248C00310122B730A9C4F9C6F8B46
:10807000ED940EC594B4D17AC9FC2D1E033DF00ACF
:1080800011A0100A47722869E7410351A50C132873
:1080900028A02F59E7400B3D5C04825CA013F73AFF
:1080A000A01C130558E25943514338C162076207C7
:1080B000394452074ABA0619801727413440054906
:1080C000C552060415441D6E041C153124290439BB
:1080D0008618C218A2314528E26289732B6AC93614
:1080E000081C0AA53144522841E63965C808180C15
:1080F00048520772EA62898BCD8BAD8428098B9434
:108100002EAC90A42E61764E079C0B2D62052DB2ED
:108110000521A025404008288228C251C68BA02DE9
:108120007E077E7C42061C09199306A30459235935
:108130001E0815403EE60E0B2EE6180B2D8A081081
:108140000F41A441A451E649C55A465A675A260A26
:108150001FE531F4091C09314420E3188220A200F4
:108160000A140A23732B836C836B6AA9681C04842A
:10817000314432082685401C0849E66ACA62689381
:1081800002051D6604140A8C83EDA4B0B4F16A479D
:108190002A1D1E0C45402D26033361C6A0C3276A45
:1081A000A0A25CA01007EEF992E6A2E4A01C064390
:1081B0005164516430061DAE0B2331430415DC14A9
:1081C00010C54164522651E55A466A8762876AC8DB
:1081D0004811BA140A41C52924314418A220941028
:1081E0000F41648B8C93CD9C0E8B6C6A8849E6BCE6
:1081F000100843398449E66289021C08687B0A7BBF
:108200004B8BCDA8051C06ED734A83AC24031E4B93
:1082100096062E06E8061C0561856A072C0E12C616
:10822000A01202A05228A01C06A68BADFFDE960568
:108230005E5C2003325CA01C06D892E5A2E45C09D7
:108240001008235964494330E2A01404442902244D
:10825000116A2540140D5A475A266A677AE97B2924
:108260006A87461D1205134185A2141A2320C228CD
:10827000E228C149E593CDA42EA44EA40E832A6A18
:1082800088312239A5421C0F846B0A836C62678394
:108290004B7B0A8BAC73D2081F62C90A0514066BAC
:1082A0009C0E6A27361EC6F00A2E85F40A25E610B3
:1082B000074923518469E7A02281A01F838D6004B0
:1082C000627DA04D400631A052C3A024042330E2B9
:1082D000041F28E2FC0C2D8E0A100CA449C562472D
:1082E0006A6772C87B09A02C08A7624662885A2672
:1082F00034031E31B00921A01C0B62679C0DA42E13
:10830000AC4EA40DE4041EE94603157A1405398425
:108310006AE938122AA018062A8B8C732A9E2C0828
:108320008862A86AC993CDB20F2DD20F1D5C0B2DA8
:10833000EA0D1DC2081C0461E651460F1361E7A057
:108340001C04A24985C0036EDE3E0631A01D6A09E9
:108350008007E6B892E69AA3A01729021C3EE2EA3B
:108360000430076341845205629E1C128B4A8B4A7B
:108370007AE86A8772C962475A2749C631B20A1C2D
:108380001930E2416462479BECAC6FAC2EA3EDA3C5
:10839000CD9BCD6AA849A531432E051C102A9C2EE1
:1083A0008BAB8BAC7B0993ED7309626786062C0857
:1083B000266288832B8B2B560B5DD40F210A140663
:1083C000CA6A07518540100507288120A01DA00515
:1083D00096BE40223CA05407DE7793069A83E03293
:1083E00044A02D9C0D1203A0100E4341635A066A4F
:1083F00067830983098B6BA01806E972A772C88A84
:10840000280667416431030A4C1351C56A879BED06
:10841000A3EDB44EAC0DA3EDAC2E834A8804100D31
:108420008BAC9C4E8BAB9C0D7B099C2ED22404679D
:1084300052268834057AEA7268E225E425E61102BC
:1084400015E02D680A5004E72061A045E03D400B8F
:1084500023DF1BA65409DE5692E692625122402287
:10846000C19E1720E2E21004023123A02404057209
:10847000C83C1413938B8B2982E97AC87AC872A8F6
:108480005A0649843902CA100A435A06832A93AC11
:10849000AC2D02120D0620162E93AC62474163628A
:1084A000479C4EA46E8B8B9C0D93CB9C2DA01C04E3
:1084B0005A264906042C0772C97AC982EAEA061DBF
:1084C000920A1DEE0F1D58042E2794032369E7A07E
:1084D00015E01C04659C2F200325381DC4031DC214
:1084E0000D32FAA020043692C5A01DC2031C04441C
:1084F0004903680C32E2A012C2A02202A0240D831C
:1085000009938B936A9BAB8B298B294A141772A80A
:1085100051A45A0630C149A4416372C8832A9BCC36
:10852000A3CCAC2D3E19881C1193AC7AE941227280
:10853000C9B4AFB4AF93CBA46D38031C044E72C85A
:1085400068081D4005100749A56A687AC99E61023E
:108550001DD211100572485185A01D6E0411A0286E
:1085600004C249658083E75CA0298251A04202A031
:108570001320809E26C1401D2A03100C02418362F5
:1085800026834A93AB938BA024044A8B2A441C0471
:108590006A4662940C1409416339027AE97AE95A0D
:1085A0004C08ABA3ECA3ECA40D24032C13830A51B9
:1085B000638309B4B0BCF0A42CB4AFAC8EAC8F967E
:1085C000041F51E646051AC52C1E272213140B85DD
:1085D000598451445143494351102C0530A151A5B0
:1085E000680421A06005414493EFA0110624043BD8
:1085F000E71BE223D615A02350E2A01C0541022070
:1086000080CE0B21A01D300A133122A01006468B0C
:108610004A9BCB0211A421A2240F7AC862057AE9F1
:10862000496351C559E5832AF8429BA02A0C821060
:1086300011A3CD8B2A62058B2ABCD0C4F0AC8EBCB2
:10864000CFA21C06AF72E849C5E2051C05A55A0673
:1086500059BA091DBE111DAA133DDE06198C1372ED
:1086600068A61DCA1331A05008A24144940FFFBE52
:10867000A01DA20F2409E73BD6DAEF7CD5F5E01761
:108680005922E214066440E22081DE2EC2120D1D42
:108690008C0A30080241846A668B6AA015E42805BA
:1086A0008B4A8309801D080514040559C53C1A4BE3
:1086B0009810046B938BA022CCA415481419ED8B51
:1086C0002A7247936BBCAFC4F0BCCFBD0FB4CFB41C
:1086D000CF72C851C551DE1C0A49847AEA936C9363
:1086E0004C93C6032D66041F82C942141DD0111D70
:1086F000D40E22A6A0332081A01C049DDF1BFE0EF9
:1087000021A0400B5CDEFADED9EF3BD5F48AA01C39
:1087100007025143412220280515E01C04C120E135
:10872000A4055004233963A015E22986197E3D2251
:10873000031DAA06140A2682E98B2A934B936A42E8
:108740001560153E1C0AECAC0CA3CC934A7AA8D059
:108750000310108FBCAFBCEFC530BCEFB4CF7B09AA
:1087600051E59E1004C64985363E28F8094DEC14A3
:108770001DCA03176A06EA2E44C8031DC0031C0461
:10878000A13924E0061C04BDE71B980F354011A059
:108790001809F9F75BD5D38AA58A8021A02F494310
:1087A000880F11A033A128A03409418372C8938A8D
:1087B0009BAA40168A401C0C2982E87AE87AA872A3
:1087C000877AA874041C042A934A3A0325E226CB2C
:1087D000441DA4051804CC936B7E126FA07008CFC3
:1087E000C510CD50C530A016C58C3D340B2D640985
:1087F0003F720704101D0E1531A0140CA661A620AF
:108800004120813903836DE02E3B761141A0B007F2
:10881000E6FAF75BCDB3A033C120A02D06051D3EBF
:1088200013100C837AE893AB9BAB9BCB938AA0107D
:1088300004498308A05008C87AA87AA882E9A0321F
:108840004AA01ECCA00532EDA019A623B48FA01417
:108850000BC4F0CD30CD51B4EF7B29DE1EC58A06A6
:1088600031A02F69E7E2143369E6A01D3A1615140A
:108870001F23616E1051A0166C40523CA0261B4075
:108880002C0FEF5BC5728AA59263510348E2512217
:1088900080071A287C297E1D1E0324066351E48369
:1088A00049DE739BAAA032C8A042C8A019801F4A03
:1088B0009B7C0423A3ACA2239BCCA02005938BAC70
:1088C0004EA241A01C0ABCF0836A520549A44994F7
:1088D000111DDC124E27A0052E6AC20E1C04066A6A
:1088E000073C111D0005140761A659A61840404C0D
:1088F0000623836CF77C1A0335DE1ADA8030045BBA
:10890000C551A02C060240A14902C00815421FA172
:1089100028A6052DFE044F6A673E04340B9BEB939B
:10892000AB83297AC77AA7DC2287A619807629E249
:1089300030048C9BAC9C2D8A041C04ECAC6EC003F0
:1089400022D09E2008D591C5318B8A5AA02DC40310
:108950001D3C0C1D54041C102349234102410249B3
:108960002340E240E22840420B2285A01218A01FBB
:108970007B4CF8043E1BBC03221A9E3004DED9F760
:10898000A060058A4248E2A02E3164041C06C13171
:1089900022310272033EE93A04100D0CA3EC832944
:1089A000624551C451A45902400761E56A467267A5
:1089B000A21D2203164BE23C04AC9BAC80042C04A9
:1089C0004A8B29700426BC3E2C0C31D592D5B3CDF0
:1089D000B293EC5A463E061C0462685136123007C8
:1089E00059A559C559E60431061D400B10066459B6
:1089F000655985A01261A030082CF77CDF1BDF1AB7
:108A0000A0119E4007DEB9EF5BBD31A01C0548C137
:108A100048E2220D33E239A01F28C1BE062C04050E
:108A20008B8BBC061C07A40C8B296A86BC081C0E09
:108A30002659E5518359A4620562056A268C071DF3
:108A400024031D6004264B3E1C1F938C830982E87F
:108A500082E8726672667AA79BABB46EC510D5B217
:108A6000DDF3DDF4A46E6A8748051E47AC0A1E0AD2
:108A70005E041C066C830A82EAE6061EA900051C39
:108A800007486A68518449B80615402620401C04EE
:108A9000730BFFFC1351A016DA42240AB9EF3ABD5A
:108AA0001082848A224021A0300630A038E228A01B
:108AB0001E493C061D3404224DA01D3E06100A49E5
:108AC0006A876A676A466A2602153E2DC2031B7AC8
:108AD000C8841E29FC063F8CA31803128BA2110424
:108AE0001408C882C88B29AC0D40180AB2D5D3DE51
:108AF00034B4F072A82A1EA9FA081D4A143D1808B9
:108B00002EC6B20316694C1DCE161004034924A0CC
:108B100035402C093103732BF77CDEFB180311A0C1
:108B20001DFE041015D698EF3AB4F08284820151EC
:108B30002340A140E249438B4BA01010C128A03034
:108B4000E149847287AC2DB46EB44DA06C08CB8320
:108B5000497B0872A7BC03419C219E2DA20525DEFE
:108B60001DE4031EAB44032C066A8B098B09D40356
:108B7000100DAC2DBCF0D5B2DE13E655C531A01CEE
:108B80000443730ADE061DD4111E616E112D800C84
:108B90001F61A61C191DE60B500949244903618574
:108BA0005165A030050BF77DE6A01DFC04110210F5
:108BB00007D6B9EF5AACAFA01004225103CA1E0267
:108BC000020F1C06A0410230C106052C0CA14983EE
:108BD000936ABC8EB46DAC2C20061F938A1E031EB4
:108BE000C8720716C9A04EE9CA087C057AA782E8B0
:108BF000620412ECA010046A8B49A02C042A936B27
:108C0000320817BCCF401C06F3DE34D5D31007243E
:108C100006646A886A683E5D5A093D6009198C1EBF
:108C2000A62E03254071A025E05EDE1C172D400610
:108C300013F75BA02808648A22512440C2801C07D5
:108C40004902410128A07C0A1804C151A4E8153E3C
:108C500021A01D62041D60091DDE061D56041F7B38
:108C60000AEC0B16094816A7C86004099329A01F2F
:108C7000A3ECC20A1D1A0511A01E8C0C0A14064E84
:108C8000BCAFCD71421C0414DE14D4081C04436A2A
:108C9000881A0E35E015441004E659C60A15EC1E74
:108CA00059200D39802A85805005310372EAA02DA4
:108CB0001C0315DE43DEB9A01409822248E340C23A
:108CC00040C2E62FC0593E09340DE130E259E5B407
:108CD0004DB42DAC0CAB1A2D8A052DDE06180B7287
:108CE000A97B0A72A9834B7AC9862A46701DA20500
:108CF0001E6B64091C1EEC938B72A872C9832B83B4
:108D00004BA42FA40EA42EBCAFC50FD571E614E65C
:108D100014834A34191E065E041F23498E052F4012
:108D2000E28403200538C230A1041F2840740416D1
:108D3000244011A01C0530E272EA300B62FAA02F29
:108D4000CE57200331A01C040148E3C20312E2A065
:108D50001C04C1934A640E14060230E16205DE1C55
:108D6000042CABEB9C051E4A36062C04A76A263C55
:108D7000031E105A1C114C1E40301A1D2E031D0CD0
:108D80000325E221A01D1A0810057AC951C51C103F
:108D9000082030C249A58B8BA01DE2061C07DDB25E
:108DA000E6149BED680B4E88FE041D4E041EA55C68
:108DB000041FC659E4171C0662076A68491005506B
:108DC00004594451A0298051A0297E1E98200820D2
:108DD000043AA46EA01C0740A238814903460B2C1C
:108DE0000602934A4122BC0B176A46DE2DFC041989
:108DF00058140582E859A4F81C08803943186018F3
:108E000081E408158C1F6A68D60D1DC4031D9605E4
:108E10001D7A071FA40D5A091C1C26080020811862
:108E2000816ACB5A2728606A46A3CBC4CFDD92E67D
:108E300035A42E49633C0B1EEA001B1D5A041D1A63
:108E40001B1E895E041C04486207201B1E06AE051B
:108E50001E035A0C35E03C0728C27B4BF77DD80631
:108E60001D7A071DA2191004D9E6FAA014064D8236
:108E70006481E1DE100AE240C1490248E172468C99
:108E80001202526287A02EA3FE091DF8071DBC0B1B
:108E90001E847A091C0A811820206041647AEAC085
:108EA000151D2E032C058B4B938BC20D1D461312E3
:108EB000C91A180861186052076A89841006ECBC48
:108EC0008ED530A0100A14A44E4984832B518402FD
:108ED0001DAE08235985062F5165DA061E51D209A9
:108EE0001D620E4E44C00311A01E4CE0064E1B5CDA
:108EF000042D3E1A1D20081C095A9C2D82857A01DA
:108F0000305E042C0540C140C19A13100469E56A23
:108F1000D818097A88B48EAC4CA3EB821FEBA3203F
:108F2000031406936B8B6B83C41C06728872A97A38
:108F300060051DAC0B1C04A9830A3A0D1C0A4A9B50
:108F4000ACAC4FB44FA40E200D1D3C03211E100DE0
:108F5000A40EBCB0CD31EE34EE54E5F3A01C080DE8
:108F600051A47AEA5185B00392850231A21D000511
:108F7000154045E011A060058DF79CDF9E2EB922BB
:108F80001C11A018070C7A6479E130B01C1140E183
:108F900048E140609B2B61848AC948E161C45C045C
:108FA0001F4CACDE061C0AABCBABCC9B6A932A8B66
:108FB000F2041D20081288021C04A882C930063E53
:108FC000E922081E8BDC0B1E2EB4081D660E1C0445
:108FD0009BCC7A4E0D239BCD141409D572E614EE6A
:108FE00055EE34E018060D61E572687AA19E2E8573
:108FF0007A0C15401C04E340E338031664E0254076
:109000001E6CB00D5D200342D6A03004399BECA04D
:109010001E81221A1C060240C138601E1D1D041844
:109020001DCC1C26A4401D60042D80071D000A1CB9
:10903000049B6B93820C1DFC042EC9E40431021EB8
:109040000A7C0710046BA3AC9E154021A01C05B43C
:109050004EB44FB0052C0C6BA3CDAC2ED572E5F3FE
:10906000EE55C0033407A40D59C562074046A54418
:1090700042519E11A22D240831A035E02C07734CDB
:10908000EF5BD6F9D8061004DEB9D602100CDED894
:10909000F73993CB7A6471C128A01638E01DE60633
:1090A0001C06C19B8C8AE94E0B1F42BC9C051C060A
:1090B000B42CB42DABA20D12A3A01D4A092102119C
:1090C000801DB608224BA42D2A062009ABEDB42E34
:1090D000BC90BC90A211A021AC140A6FB42ECD326A
:1090E000DDB3E5D3422C0635E6148B6B6607500ED4
:1090F000410340E2410338C238A138813002540BA9
:109100002860282040E251444124401E4C740C2227
:10911000D9A01005D699D698A012B8A022AAA01559
:1091200040213A1EA1E6061C06A182C9932A100F0F
:10913000200442B42CA21005ABECABEC9E419A2863
:10914000048BA38B8C31A214064A8AE9936A3E1CD5
:109150000B0DB44EC4D0CCF1B44FAB640E21A010B3
:1091600007C4B0DD73EE15A02AF47E1C07EE567A14
:10917000A838C1520911A22D62041D60041DB80354
:109180001F6A275E041C07276A484944389A031857
:109190000749441020184180228CA0153A329902C8
:1091A0001EB9400634043A8B8A401260A012E2A035
:1091B0002C10C240A161A49BAC722640C09348BC55
:1091C0006DC203154021981C048BABABCC0321A2CC
:1091D0002004ACA3AC9E10047A879BA0140BA3AC14
:1091E000BC4ECCF0CCF1AC0DD822CCA41007CCF105
:1091F000E5B4EE159E22D3A01FE5F4F20D2006A9DA
:1092000072897ACA022D42102D40062D0C0A1102D5
:109210001243761C09C241034124100010A20F33EF
:1092200083ADA0519E51A028086A7A4471A1306193
:1092300082100538C2282002140A008AE982A88B0D
:1092400008ABEBDE1E2C02052192319A37ABABEC5A
:109250002AAB8C44057A878AC8EC1FAC2D8E0A2471
:109260000611BC8F8AE9602009B40DCCD0DD73ED06
:10927000D4A22C07DDD3DDD3D572440E3D4E041E9F
:10928000440E083223042DA80A31021240A01340D4
:10929000E3A02220A01F8BEE540E72FAA01E99E0CC
:1092A00006340C3A83497A446980306138A2E22E50
:1092B000E228081F61E534061C04C8A3CAE2061DA3
:1092C00042062524553A21A62D6E0C2C08CC8B097C
:1092D0007A66A3CC96071805934AA3EC8220088FE0
:1092E000D532ABCC8AE8201811B42ECCF1DD52E592
:1092F000B3EDF4E5F4EE15BCAF626264A281021531
:109300003E1F2449F607300638A240C249A0422039
:10931000A042D99CB1A03004812840A015E429C8FE
:109320001C0530807AA8B4102EABBE03198032CC55
:109330009E50046AA36BA41542240B82A89309A330
:10934000ACABEDA3ACD629781007C4B0B42E8AE834
:1093500016100C8BABACBC2ECCB0DD72E5B302703A
:1093600004F4A3EDA0419A5324499C1102166416FB
:109370001DD809B5E05404B9DEDA4235401DD809DC
:109380004224A01D560322A1022D2803233040A011
:109390001405AC0CB44D4029801F6BA3220351A0CF
:1093A0001DCE081D840C1DE80E2C0D596361E58B44
:1093B0002AAC0D8B0969E5C4123C1793099B2AA3BB
:1093C0006BABACB3EDBC6EC4CFD510DD92E5D482EF
:1093D000E9CA10476449E24E4486073805494441CA
:1093E0002350151819801603401D220D11A0600688
:1093F0001ACEB9D6BAA01D000A421AA02004200035
:1094000030A01D56083F3080FC032C04607247FAE0
:10941000112DC2081DE2061EAC5C04124A0221A2F4
:10942000210E1C046B8AC9A20F2EC95E1F1D8A0C57
:109430001DB20515501C044A932A6E091229C61C38
:10944000096BABCCBC4EC48FCC840C1805E5F45929
:10945000C436193C115A100560286030021D5604AC
:1094600034044028400E12A2086006A138E338E315
:10947000A05804DEFACE7C3102100698EF1972E88B
:10948000A01C04601800E21C4D960441A01C0A8038
:10949000282059A47267B42D7C0F16AB3C10064AE5
:1094A0009B299B2AA2326BA02E8BC80B1C077A87A4
:1094B00072477AA8C8033EA8A8051D26051B930974
:1094C000821C076BA36BB3ECB33C0A2C09C4AFCD71
:1094D00010EE153080F8041E4184051D200D1C047B
:1094E000E6620622181F27627A0C11061C04076226
:1094F0002872144405A230A239401006A27B8DDEEA
:10950000DAA07679401C0478EEF9D40920070461CA
:1095100040100030A04404A130A0E61D2A03180822
:10952000E130A04101B46E7C30048AA38AA0822974
:10953000A02D7409380D82A87267932AA3CC726794
:109540009B8C8A268B641405A36AABAC401C062E48
:10955000C48FC4CFC40D1E724A0D1E68EC082DB016
:109560000836A5D82C040338E24E0715DE1EE37634
:109570001B3E81080A22C2A0100528A27B6CA01203
:1095800098A0210221A811A030056AA76A03A02192
:109590002C1988100520202000021C0820284018C3
:1095A000001800DA131404CB9B69404249A01D2423
:1095B0000339801DE00322A8021D54042C04AC7A58
:1095C00088D0061D82112804CC932A021BAB8B8005
:1095D000264E3E2C06D552B48F305A05319029685C
:1095E0001D9E0A3D8603610259561EE32003454035
:1095F000F2FAA04287A01DC2191E61BA0D1660447E
:1096000020048138C3421E496E181D9A145004AAC2
:109610009B699E1C04499B49C6032D20031D080D10
:10962000119E2FC8822E0D12C89620046BB44FA035
:109630002D10052005ABCCABCCA03C0BCCCFD5116D
:10964000D5528B4A38C182053E2340061DE60C1DCB
:10965000E80652E3A41EC2161C3E81DA0421A01DB6
:1096600082112B83CE8052CEA032CEA050056266EE
:1096700069E3A016814216808019B039D01EC286D7
:109680000C400563AC2D939E41023D220315403DE5
:1096900020081F7AA8AC141C0AA46A265184936B74
:1096A000AC4F3E081DB2051D60042010CCBC0DC49B
:1096B0006ED4F0CCF0DDB3620538E19A453C41024E
:1096C00021FC20043903396811A21D5A0741A01C4E
:1096D000066118618C0FB40D240499CE583A100518
:1096E000D698CE78A07004D96246A01261022D648B
:1096F000033C04812861CE03298E1E8056111E8AE8
:10970000980323099B0415C02D2E101C05830938CE
:10971000C142032D56032EE22804290A2D64071F97
:1097200051A40C0F2D00051E0DBE031006D0CD3127
:10973000DDB4F01C04224123220631A21F4103B8EC
:10974000162E02E4111D701B1805A12861204E1D64
:1097500020031D0A1839802EC2C00313D6B9A030C9
:109760000458D677A0200C57EED8622569E35940FB
:10977000080030154221A24D5A08298A1D080417F5
:1097800062262E32099C1E4A3E041E4A40063C04B4
:10979000CD6A26E80C21FC15021C1038E3496472DE
:1097A000887AC993AC72878AE9A304071D92071DC2
:1097B00082111C05D572832AEC0F12808611884114
:1097C000501007206020602880A21004A230C23808
:1097D0001E650E102E6030031208A03F30E36004B7
:1097E0003C0A79CE38CE58CE77CE77C0033008F811
:1097F0005A0469C36181A0538120011C04180041EF
:109800005E163C09938CB4F1CD93CD72BE0D698088
:109810002A8A7E1DC2281D96251D6C291004A56963
:10982000E7041C08E6930A8AE9B44E84111DE40893
:109830001DE0061C050DC4AFC4E2151FDDF4AA0E21
:109840001E80C8113C06A5496551C69A251E4816BA
:109850000D1D180D2D220D1C0551C651A6BE083A2E
:10986000E3F212E2A010134131047BAEDEFBC659D5
:10987000CE39C638C657CE98C6A813E6B8A015E0AC
:109880001D960D15AE1C17206051C572E9AC8FD521
:10989000D4DE15C532C532B4F0A46EAC6E760F1DA1
:1098A000780519862004699329A01C0593298AC884
:1098B0001E221DB2281DB4281D46201C0982689B4B
:1098C0004BBC6FABED64041D680B1D80072F2DC4CE
:1098D0009E141C0851FF59FFDCBD73C0202C088565
:1098E0004165416530E3341911022EA2B6032738D1
:1098F000C3781D340415B41DC0032EC2C0031F2835
:10990000E3C00311A0119E100617C657C678AA140B
:109910000658E69859C340100A40186049C5CDD48E
:10992000CDB498100452C572981C0E8EB4F0AC8F52
:10993000A46E9C2D83698B49FE0E3249A22E49E408
:10994000061F9329BA031C06878AC9930A722A1034
:10995000084BA34BAB8CB3EE9E1C06CDB40EAC0DE6
:10996000AE0A2C060DBC4DCCEF3C151C13CD92FF5E
:10997000BBFFFDFFFEE6FBAD14628A41A628C3666D
:10998000162E410A171DFA041C08C338C430A33927
:1099900004381A4240A01B1820801C3A8DDED9C61C
:1099A00058C617BE17C637C637CE59CE18DE775AF7
:1099B0000459A25940DE97D615C572C552BD31ACC7
:1099C000AFB510B510ACCFA4AEA46D9C2C8BCB72F0
:1099D000E7AC6E82E8FA073DBC06210215403C0761
:1099E000E88AE98AC893E00B2DE40B1D56062C0487
:1099F0008CABEE9E0A1DB20710126EBCAED550D5D0
:109A000091B4CE8BCAACCFD635EF19A432DD041099
:109A10000CDDFFBCE698DE3793EE28A18E1006829F
:109A200030C330C2AE2D8C0321A018044028C18061
:109A300022B9A042C6A01C1437CE17DE5651C3610E
:109A4000E35960C5B3C592ACCFBD517217200AEF80
:109A5000ACCFACCEACAEA48E021C077B287B28AC6E
:109A60008E74161287A219862DD2151D880C2D8290
:109A70000C1D0A122DB2191D44101E2AC4171DDE1A
:109A80001A1D4C121C2C8EB4AEB4CEC551D5D3F6D3
:109A9000D7C551940CEED7CDB2ACCDC58FE693FFB0
:109AA00056FF98FF78FF78F737FF58FF7AFFFCD60C
:109AB00035AC0E2A60F42D2C043F28A2A0052D8081
:109AC000074004B9CE379E1C1BC636CE57D656DE8D
:109AD000355182514050E0C5B2C592B530BD30A479
:109AE0006DB50FF8192C168DACCE9C2CA48D9C2C2A
:109AF00073088349A44D5A0482E861C46E11728BC5
:109B0000022D3A152D5A1A11062E8A94142538243E
:109B100033BCEFBCEEC550BD30DE14FF9AD615D66F
:109B200015FFDBFFDAE6B4C56EACECB52DAD0DB5B7
:109B30004EB54EC5D1C612CE13BDB2EF39FFFDBD35
:109B4000531820D81D340F2E41F82C1C09104073D7
:109B50006DD699C61775251418F7C616C615BDB368
:109B6000CE14DE55E655D571E5F2CDD2B530C571CE
:109B7000D42C188EBD10ACAEACCEA4AD940B9C6DA5
:109B8000A46D73086AA6AC8E51A37A142C0559A350
:109B90007AA72C034D16121DD8154E8AEC062DC23D
:109BA0000F1D14031805AFC4CFC4781D3615140853
:109BB000D3B4F0EEB7DE56DA12BBA2100EDBFFFB19
:109BC000EF38DE95E6F7EF58FFBA0E12FC0216FDED
:109BD000F026BCF41FA4D1B2251C044CA4D2AA17B1
:109BE0001C0CBDBDB7BDF7DEFBD699BE177A2A1493
:109BF0001119DEB7D676E718EEF9D616DE35E6553A
:109C0000BD3C13ACEF9430240CAC8D8BAA834894EC
:109C10000BA48D93EBA46D836A49A3C5525A046AC1
:109C2000667286622559A36A468308A22D181741D9
:109C3000A22DF80B1C04CCC48E0E081C0630CCEFF1
:109C4000B46D76161012D3BD31EEF8D676FF9BFFB9
:109C5000DCEF7AFFDCF7DC94210411061C09F79B8A
:109C6000EF7BE75AE75A7A2D3A7B961D40031FFF98
:109C7000DD1603142B36A553E71CE71BA53294D041
:109C80008C71B5B5CE57BDB3B572C5F5D678EF3B7F
:109C9000BDB4C5F4B4EFA46D93EB8BCA93CB7BD268
:109CA000140762456AC67B28E814166D93EC41419F
:109CB0009C0DB4F0414159E4620559C451A351834C
:109CC000462DE8062DC80D3D8E071FABAC3E0B3C64
:109CD00004D0D5316A151010EBBD0FACEFDEB6EF36
:109CE00018EF7AF79BF7BC0411A63005FFFCF79A32
:109CF00010200E7BF7BBF77BEF5AEF5AE6F9E71916
:109D00002211BE42BBA61C0FF77CA4F2B552C5D2ED
:109D1000A4EFD6B9FFDFE0061C28B8B5B5FFFE9466
:109D2000D294B1B5F6B5F5AC8D9C0B93EB7B695A2B
:109D30000472E772A77B0873085A44940CB4EF933B
:109D4000AB401B1C0AA3B510B4AF72A751C4781B5B
:109D50001C0A835183410159C47AA75C0E2D2C0D36
:109D60001DB20D1D600E3804B0C4D08A1E6A881B57
:109D70002408CFD614E6F7E718CA23EF5A941EFF3B
:109D8000442A119815EA318C32DC1610059ADEB798
:109D9000E7C421021405F7BBEF9B4C1C10FEFF9C8F
:109DA000DEB7E6B4BD908C6FBDD6C616E0101C10B1
:109DB000DAAD75A574AD95DF5BF7FE9C2B9C0BAC03
:109DC000031C054849A272221A1C1572C762865AE2
:109DD00045838AACAE9C0C8B6A62665A059C2D3218
:109DE0001D1C05EC834A620C082C0D496338E138D0
:109DF000E149426205728708191D26081A05001CF0
:109E000008A77AE89BEDBCF1DC05140C76F77AFF25
:109E1000BBF7BAEF59EF39D02C045BFFBD600413D8
:109E2000E7598A26DBF011A21A39601006D7D696B8
:109E3000D6B6064005B7E759E7C81414DDE6D8B52D
:109E400071A4F0AD74C6369CB0C5D4D637C5D6EA79
:109E5000200699B5F6A573A02C0772E673077B4917
:109E6000B2031C1F72E762866AE793EBB4CFA42D9E
:109E70008B6A8BAB49C349C39C0CB4F0B4D0A46FBC
:109E80008B8B04121EC8CC171EE470181008A3494F
:109E90008351C462269E1008C78B89ACAFCD939EB8
:109EA000100436EF199814109AF7DBF77AE738E6C2
:109EB000F8EF3AF79CF7BC42253E1004FCEF7B0C10
:109EC00015D41534140A7AE718F79AE718DEF7FC68
:109ED000125930267BEE2C0B946F8C4E94B19D1250
:109EE000A5111E251C189CB1A533D6D99D128470CE
:109EF0009C0A940A62655A248BCB836A7BB4031252
:109F000083A81F940C06051C084DAC6E9C4D83AABB
:109F1000261D1C06C36AC793CC0E21126E0214269E
:109F20004D9C2D9BEC9BEC9C2DA44EACAFC532CD33
:109F3000B3D5F3C591CDD3CD92D614D614EF39EF66
:109F400079F7DAF7BAC01E79BA0316D7482E791A0C
:109F5000031FE7191E031F7AF7300315E211A01043
:109F600009CE54C614CE34DE9628280439E73AAC1C
:109F70001D44031C0FDDC5F69D33E79CD6B9BDB566
:109F8000B574E6422E1BAD9484180A918BA98BA957
:109F900093EB83897E3EE8AC171C04E77308CC037F
:109FA0001FAEAC720518109C2C836993CA8B8983F1
:109FB0006972E862666A9E10058329834926122821
:109FC000181ECB28051C086EACCFB50FB52F3B2D46
:109FD000200891D634DE75EF38A01C0DE758FFDA63
:109FE000E738DEB6E737F7995A042EBBBC031FFFEC
:109FF000BCF22F2DD2034EDB780413E7172C240478
:10A0000018E6D7661DD2031C049AFFDB50311C06EC
:10A01000FFEF9C84705A1814183BDE98E719AD3294
:10A02000A5119CD1D6989C2C93CA7B488BCB4161BF
:10A03000AA2004AA7B08021E938C031009B4AEA4C4
:10A040004C93EA8B69021E482808128904100A6999
:10A05000832883087AE772C72431A21EACCE05108C
:10A060000DB50FBD70BD50CDD2C5D2D654A01004D1
:10A0700059EF587C1658442638C215CA2EBAC20366
:10A0800015E0167AFA25DC140438D69656102EDB25
:10A09000E718CE55E6F7DEB6CE96E739DF18EF5A69
:10A0A000FF9DFFBED6B99CD0AD10C5B2DEB7C5D3FB
:10A0B000EED6DE34BD72AD31A46D8B89A01C04AA2E
:10A0C00093EBC603140A2883498B8A83499C0B406F
:10A0D00014046D9BEA3C10066893A99389A221A6FB
:10A0E00011AC1DCE1C12CA06112E2F9C0B2A051571
:10A0F0003C100470C5B10211A017CE3316180437F6
:10A10000F7795C240617E738CE54442964296C4952
:10A110006A2D6E041407FFFBF79AE6F8DA11A81C03
:10A120001CD675D695DEF7D6D7CE76E719FFDDD6E5
:10A130009994D19CD0B571B571E6F8D698051C07F5
:10A14000D5F3A4CFA4D0700714066D940B72E7C4A6
:10A15000240AE76AA67B4983898348401007BD2FFC
:10A16000ACAD9C0BA01289A22102168944119A1051
:10A17000049BCA9B9C15DC14146DA48CB4CEBD4FFB
:10A18000C570CDD1CDD2CDF2CE13D674383679404C
:10A19000140538FFBACE4E1C05BDD2DED6CA08164D
:10A1A000FC2E180839DED8EF7ADEF8921E592E03FD
:10A1B0002C06BBDEF7EF59440313DED7CA14115641
:10A1C000E6F9E6D9EF5C840F94F29D1294D09DD805
:10A1D0001C19B593A4F0C5F4C6358C6FB50F83AACE
:10A1E0009C2C9C6D8BCB7B698BAAD6061016C77BEB
:10A1F000489C2CBD50BD2FB4CE9C2B93CA9BCA9CAF
:10A200000B9BEA0212CAA81006CAA42BA44C9614EF
:10A21000040FBD0F381291041270A215402408CE0D
:10A2200013CDF3DE95EFDA4C1279F799D695EF5806
:10A23000DED7FFDACE54CE34EF38A60315EE2ED794
:10A24000F204398016BB461EBB0A0512D7841C20B7
:10A2500014D676BDB3C5F5CE78FFFEA574E77C8C29
:10A26000B19D5394D2B5D5DEFAAD7394F1CED91E1B
:10A27000082C0410A48E74071C07ACEF9C6D9C4C3A
:10A280007E0720044CACCE7C35421D1E0513A44C29
:10A290009620042BA44B0A13B4CD9A10084FBD2F5F
:10A2A000BD2FC5900235DC23CDD1A01805CE33E6F5
:10A2B000D6801C0458DED616031C0C38F779CE5510
:10A2C000D6B6D695BDF3B0051EFB140511A4310218
:10A2D0001DE2031007EF59E6F8F7BAA21404BAEF2B
:10A2E00079E01C0695D655D6758E041C1A9BA5746C
:10A2F000B5D69D34D6DAF7BEEF9DA555DF1B8C7021
:10A3000095129D73BD51BE0811042DFC091FBD504F
:10A310008E032E303008151E100C90BD4FB50EACBC
:10A320008CAC8CB4CD96160E503004CDB4EE9A1190
:10A330001C1805C570D612781C0690CDD1D6121CFB
:10A340000319802405DE75E717DE1D100316792C2E
:10A350001C04B6CE75EC06140438C5F34022BA8E40
:10A360001D18031EB6DE031699DA12790E154E116A
:10A37000101D4E031C09DED6D675CE34CE554603CD
:10A380002F7B7CE6291C095CA534EF9EB5D7EF3006
:10A3900021140F73EE9533BD71C592BD91BD91CD62
:10A3A000D2D412910E12B20836502015BE1004AC51
:10A3B000CDAC9621982408C54FB4EEB50EBD3C1522
:10A3C000D63005B52FCDB1A81807D1D633D613C5D1
:10A3D0008027DEB5361FEF589E0339861C05F79996
:10A3E000C5F300033675EC1C0AF7F799FFDAEF584E
:10A3F000EF38B2031C04D6DED6860418049AEF990F
:10A40000081C0AD7CE95CE95D695CE55B2032C060C
:10A41000D2B551840DFE1D197E1C04D6AD54EE1F1D
:10A4200010063C84718CB2901C0471BD91260434DA
:10A430000671B530AD0F403952254012BD9413B4AA
:10A44000ED96119813C5909E222F14110221A0227F
:10A45000D19E13CDF20415401C05CE12D654B6037E
:10A460001DC00327EF592211A6200A38D675DED663
:10A47000CE34D6959C1DF40611A617E6F75C1E1780
:10A480001A0325F41C04FBEF7984042C0559D6D754
:10A49000DFCA031C1055EF18DE76B57373ACF79D59
:10A4A000BDF6D67922301408BEB5967C109D3432A4
:10A4B0005406B1CDF3BD7140153C31881526110805
:10A4C00040062EA48CACCD1035F02DEC04464F4048
:10A4D0002DF6041405C590D612401C0453CDF2BCD1
:10A4E000031DB40315262008BAE717DED7F7BA8A8A
:10A4F0001C08B591D654E6F7D626061DC2033EBA0F
:10A50000FE093AFB881DE00619882E5936081C05FD
:10A51000EF9AD6F78C072C05F7EF9AB556361C093B
:10A52000748C70BDF7CE79E60C0A1D3E061006F25B
:10A530007C30C679961D8A0319741008B1BD50ACE1
:10A54000EEAD0EA24E4F9803196E24040EACCD3A18
:10A5500015CC129020324F962102199A11021C0636
:10A560000FB54FCE125A042712C5DE2C0437F778E8
:10A57000BE031BFFBA781C0458BDD3C406140413D1
:10A58000D6543E100479DED7B22C0479F77A9C07B2
:10A590002D6E041D68042ED8F2061D4A08229BAEBB
:10A5A0001D9C05141EFBD6B7A554CE799CD28C50A9
:10A5B0009CF4DEDBB595BDD6A57394D1A5959D55CC
:10A5C000D634082F91B502062791C540151C317E5F
:10A5D0002C0A0EB52EBD2EACADB52EE20421A01670
:10A5E000B54016B53E15DE31AA112E1670E01C06D8
:10A5F000B1CE33DE7498051C0699FFFAF7B93E0612
:10A600001DC4031C04E717D6EC062C0FBDB2E6F6FA
:10A61000C5F3BDB2D696F759DEB702034DAA0A2D8F
:10A62000440B154021AE1D4A081C09FFBCF77CFFF6
:10A63000BCDEF9AE0A181AFF9D548CD2E7BDFFFFAD
:10A64000DED9AD538C70F7DDFFFFA574D614C5D2EB
:10A65000822D1403119C37ACEED86D3E042DDE0420
:10A660001D48041FCDF284051EF2DE03198011A2DD
:10A6700011C4256841A621A43C05D674E716FA0446
:10A680001DA00323F799A2197C2EB65406155A1E55
:10A69000B6A0031C0454BDD3E20B1FBBEFA6051CE0
:10A6A00007D697BDB4D6B7860C3EFC4E062EDCDE30
:10A6B0000D1C13F77BCE36AD73A57494D274307C29
:10A6C00071EFBDFFFEC40A2E7B04231C0B7BEDD66D
:10A6D00055DE55C5B2A4CE2603198A351E31762D16
:10A6E000D80443CDD1A027D5F2C6297235E4257010
:10A6F0001DCA0335681E2F2A03297E3C0437FFB983
:10A70000A2032A58F625E41C09E717BDB2DEB5C539
:10A71000F3140D2C0491B571E6061C09DEF8C6157C
:10A720007BEC6B6A4809240C6E9CCFAD10BDB3F76F
:10A7300059FF9A4E1C05E6F9D697B60A1C1E1994C5
:10A74000B194F273EF73CEB595948FFFFCDEF79C56
:10A75000AF8BECD635C5D3D614CE14BC031E50CC6B
:10A76000031E70640425BA1DA6031D38031AF29C4B
:10A77000354039802D32062290BA23C5D11832CD0A
:10A78000061805BD91D6747E5F17FF720521A619C4
:10A79000741408B6D654BD91E6D64212F39E1C1A24
:10A7A00099EF59C5F4B5B3630952875AE85AC8629C
:10A7B000E8840D9C8F9C8EA4AF0E081C0CF4D697D9
:10A7C000F77BC5D4CE56D6773C0B1DFA271C0B9CC5
:10A7D000F2A532B572B592AD30FA0E1FD0CE8A090D
:10A7E0001C04D635CEBE0915901EB2860811F03570
:10A7F0002A1D9E0335EC1C0470BD6F84052C04F2E9
:10A80000D6327604210E16BDFC1FAD0E0E05322F7A
:10A810001E4C0491D6531E032BF7787C1D20061D79
:10A82000E8042D40091D9C05100E17AD2FB550DE14
:10A8300096DED7AD30BDD39E1C12675AC952885AD6
:10A84000A962E983CC8C2D8C2DACF03C061E760AD7
:10A85000071814BCC615A5129CF173ADCE98BE1690
:10A86000A552BD91EEF6B4100C97EED9DE7883CCEC
:10A87000C5B3CE15A01C0435D635740E1406B6DE4D
:10A8800075DE5494240450ACCEEC1FACEE4C041E88
:10A890000E1E031EB0A6034DEE04198C25EC37C521
:10A8A000D1522C0AD2D674E6F6E6F6E73722031F19
:10A8B000EF78BA082E3788051D7A071C0654BDB2FA
:10A8C000CE34F40C100C55D655C614DEB77BCC52E2
:10A8D000A89E1C1AA95AC95AEA630A83ED946E8C81
:10A8E0000DA4CFC5D48C2DDEB7F79BD67798312831
:10A8F0000A94A5538C6FAD739CF0521C05F739EF89
:10A900001AA61E2C185B39836B0AB573C615C5D4FD
:10A910009C8F7B8BBDB3DE96E6D6D654FE0F2D2CD6
:10A9200006396821A03ED1D00656D1F43EB1960436
:10A930001DD6061C07D654DED6E75778052E99BCDF
:10A94000031D9E05300437EF57AA1D9E052C07B541
:10A9500091C613B5715C071007F77AA51152689A72
:10A9600012CA022018EA5B0B634C8C4F8C2D942D7D
:10A97000A4CFB572A511CE35EEF8F73A8C1C11CEE6
:10A9800077AD9394D1B5B3CE34C5D3BDD5AD746492
:10A99000041EF12633100FE641E54A2642063143F4
:10A9A00020E13983C5A21DB0061C04F3C57040091F
:10A9B0001ECDA8051E6F62041E905406319C1D70AA
:10A9C000072E33740749861006C5D2C613CEA211CE
:10A9D000021C08B5E716FFFAEF37D009254E1C0414
:10A9E00017DEB5B8032695421408B551B592B59354
:10A9F0004ADA300D5AEA62EB5ACB632B5B0B6B6D74
:10AA0000A01C064DA4AFD696CE032C0456E6B7661E
:10AA1000041D021E1C17F8C656A5948CB0AD529C9E
:10AA2000B0842F73CE8CD18CF152684A18382F39EC
:10AA3000C656391C09398421017B6BE6B774041CA6
:10AA400006B2CDF2D5F2E2091AEE7035CC2C05D65D
:10AA500033BD708E054C06DE73CDF1D6CC031C08D9
:10AA600091CE33CE33D695B80815D41D1E082E9935
:10AA70005E072DC4081D28082A5974340DC5D3C596
:10AA8000F3AD51AD518C4E5AA938120BA21FEB6396
:10AA9000BE344B9CD1801FCE368E0F1E9330101CBF
:10AAA0001E19FFFE7C4F9D32ADD584D2B5F6C63758
:10AAB000D678AD549CF294D2849052695AAABE3191
:10AAC0002DBC381DE22F2C0931633142B552CE1511
:10AAD000D40321A23DCE061ED10208196E2DE0033B
:10AAE0003D2C0B29842D72041E331809153A2405B8
:10AAF000EEF6EF16302D00051D5E071D04051D4204
:10AB0000091C06F7DEB7AD307C031E35DE091816CA
:10AB1000B462E95AC9634C632B630B630C632C6307
:10AB20004C738D9CD1821C094DAD31D656AD52BDB2
:10AB3000BC032C0FEF5BF7BEC67884B08CF2849117
:10AB4000951362271FEF1CC23A2004FECEB9A03134
:10AB5000A21628441E859A3A1DE82F13A4D0FA2C79
:10AB60000692D634D63420061D5E0C4004F2DE5424
:10AB70000C1D6E071C0433BD90C2032D940A1E12D7
:10AB80007A081233BA2EB0060A1C05C612D694D023
:10AB90000B2DFE0921A2180638B592BDB246100849
:10ABA00092BDD48C6F4A479C24042B6B4C3C197E7D
:10ABB0001C042C6BAECA061C0E2E942DAD11D6565D
:10ABC000BDF49D11C5F5F027181C7CF7FE73ED8CC4
:10ABD000D1C699FFFFD699BD95B595C638A574CE57
:10ABE000785AAB5AEB181406AA4A2841E7E61E65C4
:10ABF0003E3B1C0E43316383CCCDF4BD92DE76D652
:10AC000014400A2C0413C591200B399626D2E42F48
:10AC1000D633B8031FCE535C0A3674FA200A90D696
:10AC200053EF16F778FFFAA02D1E081C09CE75BD4C
:10AC3000D2C5D3B550C8041406734A475ACA361051
:10AC4000062B634C6B6D9C166D401C0CEF9CD283E5
:10AC5000ED9C6FB573CE36B4081C066AC5D4DE977A
:10AC60001E3F16DE421C0E90C679D6DAD679AD3478
:10AC7000B5B6CE9AAE0A1004FA5ACB0211D81C0807
:10AC80005AAA422839E731F6391DA43A2C0B633908
:10AC9000A462E9BD73CE15D672041E95FC0C2C047B
:10ACA00013DE75020D16C5D6153E1D6804219C27BE
:10ACB000DEB54025EE1EC5C2082D4E0E2BE73782AD
:10ACC0001D9E0A1DBA08140BCE14A4CFBDB3840E6A
:10ACD0004A483C419A14040C6B4DE810066C73AE64
:10ACE000A533A01C0E4FC5B4BD94B553AD12C5B469
:10ACF000E6D8C8121C089CFFDDAD948490D6101CC9
:10AD00000CDDFFDEDEDBDEFBCEBACEDAF2031C0AA0
:10AD1000EB6B4C630B5ACB528AA63312E7A01D9CF7
:10AD20003A1DC4381006C55A87A4F1A21C0575E661
:10AD3000B6E64C071D6C0A1C0454D65412031D8E33
:10AD40000A2D180315CC2E95320B1DA00B4C0E545A
:10AD5000BDB1BDD2C612E6F6D6B5E6F6B8031D54AF
:10AD600013280C18E6F7B572AD324A6852AA76136A
:10AD70006B6D02124D6A11022373CFA01C1BA490AD
:10AD8000BD94CE16B553BD73C5B4CE16F75BF77C34
:10AD9000F79CEF7B84907C4F6609300AF6A555AD91
:10ADA000D674308CF3A014046D6B8D422006CA4A11
:10ADB000683A07A01231A01D783911A41C05A5110D
:10ADC000D635460F1C04D7E6F7000D4275A6119C38
:10ADD0002E95BC0B3DD6131DD8131D5C073D720C80
:10ADE0003D8E0F1404DBEF58DE140E34DEB7DEB7F1
:10ADF000FFBBCE566B2A52899E2D160330064D6B33
:10AE00008E738EA662ADA02007CE16C5D5B573A2EF
:10AE10003C05D657EF1AF4401817FEADB5A5749C43
:10AE2000F29D339D558D3484F385135AEA5AEA6BAB
:10AE30001A25441DF43925E41A858615442D843CD1
:10AE40001C0741E6B552DEB662142DCC0E1DCC0CAB
:10AE50003D120B1DB60B1DF6041DE6111DC8061D87
:10AE60008A121C05E718E718F2111DEA09111C1DCA
:10AE70002C061FC5F4A20A1E9BA80816D5DC26685E
:10AE8000A01540422DA01404738E630C20117C0F7A
:10AE9000A5348C0EAD11CDF6CE16AD329CB0A02DE2
:10AEA000123F1D984110127CFFFE9D139CF38CB144
:10AEB00084D29D9595348CF2A012CAA0478D73421E
:10AEC00021A21DC8031F39A6A8351E85BA3A1C0742
:10AED000854A26BDD3DE10092DF4071DD00E1AB603
:10AEE0005C200434EF599C2D1E101D20101D4013B2
:10AEF0001D640A4E593A101FE6D79A151ED7201224
:10AF00001C0619DEB8A4F27E3B2FA95AF2041404E1
:10AF10000C5B0C40226DA01C0B73AE73CE7C10A595
:10AF20003483CD2604153E1C09AD11A4D08C0ECE61
:10AF300036522C2E7B783E1C09EFDED6FAC6788C72
:10AF400091840C2C0674B5B58CB174061C076B6C1F
:10AF5000738D73AD640348060B5ACA42288631A02C
:10AF60001EA6BA051C05C55AA8CE8C172DDE041DD9
:10AF70001E061ED6B20B1F75D6F2071FE6F7260E69
:10AF80004D80121D82141D240B1D360B1D660E2EC6
:10AF900013B20D1D2E0E1C045ABDD5B803140CEAB5
:10AFA00052CA5B0B5AEB5B0C5AECE0126E9C16AE6D
:10AFB0000A1C14EE7C10AD544A06AD11BD74B55395
:10AFC000A4D09C4E9C8FC2032DF4401E3B822A1CB1
:10AFD0000C7CEFDDDF1BCE588C50C616BC141E5BFC
:10AFE00014071FAA6B3205113A164C422EEBD83BC0
:10AFF0001D2803319E1DCE031102140539A5738B44
:10B00000421E5954161DD8091D24061FD7FFE213EE
:10B010001DF40C219A2E59400E1DAC1215F81D6E10
:10B02000071D72071114180839D697CE565AE97AB7
:10B0300025DC1E2B5C042E0C2203140773AE7BCF81
:10B040007BCF3E200C2F84509CF3944EBDB3AD3289
:10B05000A01D84041E52F4131297A01E1A9C141CE7
:10B0600008D9E73BE6DAEF1B540B1406D9D656D6BF
:10B07000368052CAA01DFA391D220735421DCA0367
:10B0800045E61D9C3C1E39203A1F840DD2232E5AC2
:10B09000E4091D780A1C06D2C614BDF37A0A2A55A3
:10B0A0008E410212C5101C05BDB1CE54400B1D1AB5
:10B0B000151405CE56630ADA2EEACC06310225E0D5
:10B0C000420CA01C0F7BEF7C0F8450A513AD32AC5B
:10B0D000F0A4F15E041632481A93B42C08B7D6B81F
:10B0E000BD94DEB85C271C07CE37F75CF75B7E1596
:10B0F0002004BCFF7B92236B2CA06F738D680437F8
:10B100004A48E63EC60E0513A631A61C074A267B12
:10B11000ACD697EE0A2D86171EBB400E1C05B6D680
:10B12000B6B5180B1FBD91A00E12B2065DBE12255A
:10B130003E5005DEF97BCD9E620CA015E020040C8C
:10B14000738E9E1C0B7BCE7C0F94B29CD2B5329C2E
:10B15000121C0ED0A512AD33B574BDB5C5F5C6151C
:10B16000181C1C0457D677FC181C06B9E6DAFFBD7C
:10B17000CA442C063BE6D9F73BA00515402D5C03DD
:10B180001E8D3E05114E1C045ACA524E061E420A1E
:10B190003F1DDA3D46A6441C0742064A26736B282B
:10B1A000074E5A280E210225D81DAA081D40181343
:10B1B000FF79BA1DF61127F77AA61F8C4F6E071D6F
:10B1C000A60835D62A2D3611A02EEBC00310097B18
:10B1D000F0843084108430A01EF2241514106FA463
:10B1E000F1A4F1A512BDB5AD33BDB5C6363C1C0406
:10B1F00098CE167E252C0598E71AF72A441D1205CD
:10B200007BE6FA8048048D7BAE8425521C0552698A
:10B210004A4892071EC7520636A6EA16C6F42C06FE
:10B22000265AC8B57362163D34182DE0185EFCF03E
:10B2300011210E3C0EDCF7BCEF3AD6B87BCD630A89
:10B24000630BCA061E8DB4032E4D5A0419801DF4DB
:10B2500009366B401C0B84508C709CD2A512A4F153
:10B26000E20B1E8F3C06140CD5AD12B574B573C538
:10B27000D5DEB83C1F77E61E441FE6F9AA051C047C
:10B280003AEF3BB4051D2003114E6A4C821D7E3CF3
:10B2900041A24DD40812E7A225E011061D5C402C06
:10B2A0000E2752674A4683EDC5F4F73AF73AE41899
:10B2B0001D9C172C04DCFFBC40182D700D2C05E7DD
:10B2C0003ABDD5A4083F6B6C50051D4A042E6B9007
:10B2D00005268E961F6B4CF609100C8D7C107C1089
:10B2E0008C719CD2AD339E2004B08C2E9E1DA00587
:10B2F0001B73AD861C05CE36D6771C2B1C06D8E6F4
:10B30000F9EF3A7E2A14041AF75B4019842DBC0722
:10B310002DD605398251A0198621A23269A05D0E71
:10B32000051D68431E47020B1C08A84A265A87942D
:10B330004E7A083F36E6660F219C1D5C231C06579B
:10B34000A512634BBA0B1D6A071D42042004CE737D
:10B35000CF8C1D8C0D3EEF54042DA0061E6D2003D6
:10B360001004EF8430A01C06F2AD338C4F2008246B
:10B3700012B0BD94D6579CB0A4D1AD11AD32BDB4BE
:10B38000DEB8801DC0031E1910141DA03231021E2C
:10B390007C3E05354051A42D240339D43DD40815F5
:10B3A000E44D6E0429841F4A28DC0C1D12381C0D44
:10B3B00052678C0D838B7B6A83EC948F26091C0665
:10B3C000B08C4F6B6B5A0C19741D5A0712AD9C2030
:10B3D0000CCE84918CB28C9284517C10043F7BEF14
:10B3E000F6041DFC04397A16D3401C0A5362E96244
:10B3F000E9B552B55360041004D1A4D0A01612E2EE
:10B4000016F5DC1EB86A0E1EB826031C0636CE36AC
:10B41000FF9CC4031ABD1A2E2C903F153A254621D5
:10B42000EC5C044C6B2C28035E89CA032D4E061E6F
:10B430006538421E89080B1C0AA85A879C4E940D39
:10B44000942E020B1C040D5AC8E44210068852A91F
:10B4500052CA3C3016CE6BCE6BAE7C30B5D7CE9A8E
:10B46000C67AADB79D359D148CB3A61C0A308430C6
:10B470007C0F7C0F8C921A031C0AF3A4F39CD27BE2
:10B48000AC944FFA041004539C6F022290042540A0
:10B490001FC6167E201DC2031FDED97E0C1C08129B
:10B4A000FFBDA4F2BDB5D40A21023DA8043D480663
:10B4B000354421A41F62EBC8031F694ACC423DCC2E
:10B4C000031C04A639E74E072EC91E0E1156200490
:10B4D0004EACD0F82007738B632A5B0A9E21A02C08
:10B4E0001D73EF9514C67AC6BBCEBBCEDBC69ABE23
:10B4F00059BE18B5D7AD76A53594D394B2C52B1CDB
:10B500000794B394D3A514BA0B1C0CB17BCD8C0E4D
:10B510008C2EA4B0942ECA3C124FA22E900C0A2C52
:10B5200005F75BD6985E1D2C05C616E71ABE0D1CE6
:10B5300005FFFE6B0AD80A3E2B7A0B3A0B3C153EF0
:10B540001D6804354C1D920B360B442E695C0B3183
:10B55000A01E48DA03100A6862E9ACD0ACF0B5313D
:10B56000042C0652840D6B4B22061D0409200C8E00
:10B570007C30A596CEBBC69AC69A9E11061008BB13
:10B58000CE9ABE39BE18A61EB6B01A100E3494F369
:10B5900094D39CF39CF3AD3483EE022408ED8C0E1F
:10B5A000944F940E421294A22C05B553CE15C203AB
:10B5B00025DA2D48061DA81B21A21E9C3E0A3DB877
:10B5C0000C15D42E0BEA0B2D0E0A498E1C046B6C45
:10B5D0006376033D6C041E49A8441D18441C1742A1
:10B5E00048632C52886B0AA48FA48FBD51BD52BDF5
:10B5F00093946F7BEE5A0810084C6BAE6BAEADB7F0
:10B6000096167A40169B3A100839C69AB5F7B5F8DF
:10B610009E1F39B54D4312ADA214109D14A5359C43
:10B62000F3A534AD547BAD7BAC834214098BEE7B28
:10B630006B9C4F942E461DAC3E29803DC6032ED8F0
:10B64000DE331D60042E3A2003180521234A48707A
:10B6500015421DBE0838066942285289921E4C26A2
:10B660000425423E4CCA032D9E0C1004E741E71C02
:10B670001E2CDC421C042AA4B0721F100472B531C7
:10B68000A0280690842F7BCFFE20079D35C679C663
:10B69000599A119212F8961404D7B5F8DE1008964C
:10B6A000A535A555A5549E1540369C421C05A513ED
:10B6B000736C5A3D1408AD8C0E52276AEA3E120E86
:10B6C000A01E6F6C041D860C1DE0061FD8EF8807B6
:10B6D000253C2DE8471FEF3B123D1C056552896252
:10B6E000840C1F52690C085C06E742285AAAD20350
:10B6F0001DCA033D160A1D3E0D2D56452F39E7E2A2
:10B7000008240552687B6BDE1C0BD614BD93CE1546
:10B7100094708C50A0031C04CEA5551403119C1CDE
:10B7200007B618B5D8ADD71C03180455A555761E15
:10B73000D34E042006F48C928C9102100594B28CA6
:10B7400071061C08929CF36B2B7B8CFC3D1D2441E5
:10B750001C07942F940E8BED4A3F1C044FB5320802
:10B760000F1FF9DE3E061D82071EF946062C0E77D6
:10B77000E6FAD678E6D92124294439C6460A1DD4EA
:10B78000452C086531A641E74A6974042D06051168
:10B79000A82DF0063EEB4C061C06C6528A7BCF163F
:10B7A000051C0A4883CCAD11C592DE567408140AF4
:10B7B000779CF28C507C0F9CF3C816383622389C4C
:10B7C0006C05AD969D3460042DBC032DBA032F8407
:10B7D0002FB6082DC8031C0594B2AD747E033C0639
:10B7E0002B83AD8BED1C032E2FE83F1005A4B0B5C5
:10B7F00032501D40061DC0491EB85E043E572E1231
:10B80000100AB9D678210318E310A2A62C046521EA
:10B81000240E084D06033F5ACA4A0F3E0BAA051EC6
:10B82000CA6604153E2D6A0521A01C088C2EBD7227
:10B83000CE14E6C20B1FDEB8460F4006F3A555B581
:10B84000D7A03FA576560416343212929A2E100CC9
:10B85000052D920A2DFE041F6B8DFA091DE0061CB2
:10B86000058C71AD54CA4114066C8BEE8BCDDA2574
:10B870003E12CDAA126FA02004F5DE989C1FC616BA
:10B88000441F1D444C200FC5F5BDD5D6780861086E
:10B890006110A218C3A225401D6A072C042852AAD1
:10B8A000960B3D90101EEACE082C0C89424831A51B
:10B8B0005ACA83EF528AC0031C05A4D0CE35461263
:10B8C0002C0DB6EF39DF1AC637BE38C679BE9F35A4
:10B8D0001675D81E96A40316F43C3F718496055D38
:10B8E000700C3E6D5A0E1D180D2D220D1D261A1EB0
:10B8F00071520A1F4B7BE03F15DA3404EE93EEE001
:10B900002C072EACF2C5D5E6FC311C0B36AD327BD4
:10B91000CDBDF5B594B53E0D2409CE57084008615C
:10B9200018C2E63D760C1D48041D880521A02102A1
:10B930002D86072A697A1DCC421EEE600F2DE0038A
:10B940001EA9421E1EB3700E1EB66A1E1ED9942971
:10B950003DEA041C04B5F7A5A00321021F94D3AF50
:10B96000301E30880A3EAECC0B4DF6051D9E0B15E1
:10B97000441EADC00D1E4D820C1F0B2910351C0737
:10B980007B6C83CD8BEE884522CD021E948C071CE8
:10B9900009BDB4E6B9E6D9C616C6431EB04E061EAA
:10B9A000F676091406F6D65710823E1406E32945AA
:10B9B0002965403DEC093DE8041EAA14061F894A8A
:10B9C0009C111F3A07D40D3EC6B8051E6DC80F1C4A
:10B9D00004A962C9EE0A2ED3C0151C07D696CE98CC
:10B9E000CEB9B6031C1079BE399D75ADB69D35959F
:10B9F000138CB27C30012132EFA01D520A3D700C35
:10BA00002C06AE7BCE7BCE7E07110816EF3E1D8E38
:10BA1000471C074A067B6B734BC4411C04AD8BADBE
:10BA20002E4611042FA4D1C20829761DD00D25DC85
:10BA30001EB40E0A100A57DEB818E318C3294402D0
:10BA40001E65900A3E86320B2D2A061E693A064D67
:10BA5000A60A1C06E739E76B6CE6041C056C6B2B29
:10BA6000622A031C05734BC5F4F6141ED3C01A1CBE
:10BA70000696C657ADB6B2031004F79D559E1D1429
:10BA8000033F94F36E0743CF739E11A021A84DD4BA
:10BA90000B1D20031D1E032C07840F7BCF20E3DE2C
:10BAA0004B1E6B24411C047B4B8368042C078BAD1D
:10BAB0007B6C8BCD42061C04DE98E6DA062D400630
:10BAC0001D300D1D4A0B2C05DEB8E71AFC482DF47D
:10BAD0000E453E35403D2C062DD6061DEA0B2E2781
:10BAE00056042F7BCE56061D6A041C08A942277BEC
:10BAF000ACB573F8141D16161DE00B1C06FAC638FB
:10BB0000B617B0033E14DC042ED2AC0331A0419E24
:10BB10003ECE300B1C0BCF8C517C307C50849184FA
:10BB20005C041C058C51528AA44A1E44760D1C04E8
:10BB3000A96AEA8242128DA21C088C83AC7B8C9C81
:10BB400070AE0F2E3662042FCE1628032D0A0A215E
:10BB5000023D18034686D81DD20B2D200325341E26
:10BB6000C668042E48B005153C2ECEDA082DCC034D
:10BB70002D80071C098C0DB552BD52D655121C20C4
:10BB80000655A553A53402240794D39D138C92D84F
:10BB9000777C0F3E21082D900A2D320B1C04508417
:10BBA00071D4081404928C71DE1DC2041C04294453
:10BBB00042C4482F62C9EC4410058BAD49E5A81E6C
:10BBC000AD8E112E339E0A1FCE162E171257A21DB0
:10BBD00084391DB40F1E5BA005119E1DD64A1208A4
:10BBE000043D1A0D3D1E0D1DA80511A02004486B33
:10BBF0004C9E2D980C2D10491D88121C050A9C8FF7
:10BC0000A49E051C0BCDD4BD92C5F48C7094B2A833
:10BC10002212B20226912A59763ACE742D89233106
:10BC20009E138C519821241C07B29CB2732D527024
:10BC3000032D900B14055AA95268421E0B70421E28
:10BC4000A86E471C04CD942F820715D61EE6BE357C
:10BC50001FD657C2351DE60B2DA60A112C1DBA069C
:10BC60001F4A28AA087004495289021DBA031D18E8
:10BC70000F3C046D7BCE36083E4D9C071EA9AC07D9
:10BC80001C040A9CD0F6112C0472C5D3201823ADD5
:10BC9000547C1DF6192A91642F7BEFA00951A01D39
:10BCA000060D25EC1D900A1C043194723C061DC241
:10BCB000082C059CF384102A1315A61D7A0D1F6B02
:10BCC0006CF2151D0245198410066C7B6B7B8CA0F1
:10BCD0002633E02D82071C05A4F18C2E6C0E1DB0BE
:10BCE0000A3405EF1A21032C1DF4042D4E091D20E2
:10BCF000083ECA96051DF60B3D1C043DFA104D7812
:10BD00000E25402C05736BAD11DE061DB6151C0506
:10BD1000519CAF8C12064C0594918C71A0033DACE4
:10BD2000032D880A6ECE400B2DA00A453C2C079DA2
:10BD300013A5348430A00B2C0D5ACA31A695123AA3
:10BD4000272163B59544481F7B4BA8432E2BE4065F
:10BD50001EB51A481DE0061DC60D1DB2142D200388
:10BD60001D1E031C08E71A084110A239FA071D8C92
:10BD7000104E698C0C2DDA064D040A3F73AE9C0CF4
:10BD80001D1C1333528A222289A01DEE0F1E93FE22
:10BD9000091EF0420C1650BC3650385E8D1C103D0A
:10BDA000C0104978319A22F39C14079D349D139456
:10BDB000B28E1DC40E1C194A6952EAA594A5B57429
:10BDC0000EA574A51341E6730B730A838C7B6BA2DB
:10BDD000051EF156271C0497D6576A0E1E1680259D
:10BDE0002E5762091C05E71A18C23E061FC22924F5
:10BDF000082DAA0F4DAC0A4DA00A4DEA0B4D820743
:10BE0000355E2E48C0471C08B531A4AFC5B3AC940D
:10BE10000B1DC4161E0F30042DDC032EAD340A3565
:10BE200042419C1E512A0B1ED322133E9658091DD7
:10BE3000FA091B84712C1DFE0E1D9C4A1C0E693ACA
:10BE400027A574B637CEB9A533A513740D1C040706
:10BE5000730AAC0522ADA03D1C031E77EC1F1A36F9
:10BE6000822656421C07EF3A21032103640426244C
:10BE7000E85E62F00F5D000A5D8A0C153E15FC1D40
:10BE8000720E1E28BE031E2EF60F2004AFBD72A038
:10BE90001794903C5ECE700B2D3E0B1ECFB40D1D43
:10BEA000120D5C07843194F3AD9694072C0AF7B514
:10BEB000D79D147C30636D1A052C158C30738D2141
:10BEC000441081636CC6787C2F10A110A17B8D1269
:10BED000481DD44A1C060A5A68A4B0A8141ED948A2
:10BEE0001A2297A031063C0477DEB8D4061D4C0414
:10BEF0002F422810122F4A69B40855404D54145D42
:10BF0000B20F25E01F5A88360C1C04B0ACF0CC1ED2
:10BF10001C0731A4F194908312061D18113E4DB4F4
:10BF20000D1D200629761C098C929D35AD96BE18F4
:10BF3000033A1D58061C07B5D79CD373AF9A0F1D43
:10BF4000F80E2D3C061F5AAA8E2D2C08C22944D665
:10BF500099082028481C0539A58BCEC44A2C094BCA
:10BF60006AEA5A679C70CD220D1ED876071E36E607
:10BF70000B319E1C05E6D939E68C042DCA111D0E25
:10BF80000D1D02051DCC105F52AA16033D6E0E4D0D
:10BF9000D20D25FC1D1E0D1E880809100431AD10A0
:10BFA000041C0611A4F28C2FD20F3F8E6B0E0C7363
:10BFB000634D9E1E14CE081E38A80A1C0838BE18F1
:10BFC000A596845172073AAF8E19AC1C0A9492312F
:10BFD00045188218614A4E4911A81EA232393C0404
:10BFE000C2A4D208052C084C8BCE940EBD749A05C1
:10BFF0002DC4032C05A4F17B8CF4102FDE98E804EB
:10C000001D10083DB2082D100D1D4A065C0644396E
:10C01000A65AEB22033D300D1D56142D9A0A21A07D
:10C020003D7A0C2C07B551AD319C91AC06319E1C6C
:10C03000044D634DF6042C0AAF7C1094B39D14ADEF
:10C04000B7D80B2DDA0B1C05A5757C10960C4E107D
:10C050002C03119E1C04915AAACE2C1C066120C2EE
:10C060001881B6351C04611881CA481C04C249E60F
:10C0700066471C0489734C964A1C044FBD73861294
:10C080001E5B8A111C0756B594A4F1C562092FD610
:10C090007796032DF0043D0C132D540E1D40051C06
:10C0A00005294418E31E512E89760E396035241D6A
:10C0B00048121E0AD24A1EF0561C1C06EFAD3194DF
:10C0C00070324C2D7A0F2DF6162D2E101C04AF8CCD
:10C0D00072620C1D020A1D16031EB7D40B180476DB
:10C0E0007BF09015541DD2101E71A2051C04918482
:10C0F000302C0411961310419C2E82762F2E10BCEA
:10C100003F1D18481DE80B1C08CA7B2B8BEEACD1D9
:10C1100038061ED8C4081E15842A1EB43E291C06E3
:10C12000D5CDF54207F2033D04193D06183DB20D89
:10C130002D5E1311A422C2A45E731E0921A02C053A
:10C140007B8CB532780C2D381B253E2F73CF6211B6
:10C1500025DE2D7E0F1D20082DB403100476ADB60C
:10C16000081C043584314A132D02051E50580E1D3B
:10C17000DC0B20099471294510811040A2253C1C3C
:10C180000510611061DC0911101C05082020A14078
:10C1900050120BA04D040A2004D8CE56A02DB60F85
:10C1A0002FC5B4C60621022DDC061D1E035E2B889A
:10C1B000162DCA171C046521036C081624EE3ECA0E
:10C1C000BC182C062B83CDACF17A0C1DDA1841A0DB
:10C1D0004D62113D900E2C057BF07C30720C1D8C55
:10C1E000072C0434A535400B35D81E5124221D08D8
:10C1F0000534059CD252893A19742102297E319E58
:10C20000110A1DB8421C04A228E3380C2C068D9498
:10C210004FCDF6C20311021D18192C09B552ACF10D
:10C22000A4D14227E6092D820F2DC4082F39C6CC90
:10C2300011198A3EA928072EA67A091D82042D7E8F
:10C24000091FE752BE031D282A1C04B3DE55421CF9
:10C250004EF46E074D200B1DC20315E01DBC0B36BE
:10C2600072CA1DE60E3D9E051E917C07419E1C076D
:10C27000B27B8E20A2201A0315DA1AA2801404A21F
:10C2800018A24A274010F025EA1C04811860504B80
:10C290001E0B704C1D2E1C27DED8DE1FB552FA1067
:10C2A0004C06B09C6F10A1A8081D4A091DE01A1D7C
:10C2B000840C1C04655ACA78501E2B06141D700786
:10C2C00021B63D12191DCA171F4A27460F2C0431EB
:10C2D000E6B77E071FCE56720A1DE80915F82D5ED7
:10C2E000042DFC161D22032F7BCF020D1D6A091D94
:10C2F000B20D2D4C092DFC061C0994919CD37B6D2D
:10C300003965C84C2EA21403252E3D2203297E3107
:10C310009C35F215FA2C073965942FAD12E2102DD9
:10C32000201615E01D22141C07ACF110A208619C18
:10C330000D1D221C2E3A18173EA5E2546E68E2101D
:10C34000299C1D3C081C09475A886B4A946F941A13
:10C350000D1D46231E11741F3E161C0B56EF402E5A
:10C360008D4E133E73BE151F8C51CC061ED2B208E3
:10C370001EB1560E2012719CB2A4F383AE49E74958
:10C38000C728C3184118419C1720C33E14046110EC
:10C3900081465382109E2D76042C070800736CA4EE
:10C3A000B102142FD697460615441C0953B53342E3
:10C3B0000710A2002C052D340B7D7A163C04654A2B
:10C3C00007920A3E2B56101EA93C4F1D58091C0F00
:10C3D000940D9C4EB511DE76C5D3E6B7B573AC0BA4
:10C3E0003FCF6B3C133D4C0952CF021C04EF94929B
:10C3F000100A16D244229102319E1406A66AEA4916
:10C40000E63E1D88321DB0571E2460043D5C0411B9
:10C410000251AE100620C320E320B41C0531449C19
:10C42000B128121297023C0498DE97C2031C0AF549
:10C430004A4939C729240861662E5C04A229652E61
:10C44000032D3E151E6972172D800D1F0B6B064CB8
:10C450001A9C0A2C108BEC942DACD0CDF4E6B7CD01
:10C46000F4A5117B2A181D9A0F1F73AE7414525134
:10C47000A21DE0132DC21011A01D3A2A15DA1C06C8
:10C48000D28C0F49A6684A1C0548394328BA3E2F6A
:10C490003924024C1D884915E015EA1D264D154E1C
:10C4A0004004C228E39E1D24542C04608C0E2812E4
:10C4B0001ED620032FC5F5840C3FC5D544131D504F
:10C4C000181D28081E81BF351E00CE0D1EE3F20B7D
:10C4D0002D500B2C06C752AA62EB38541C0D9C70D1
:10C4E000944E8BEC8BCB942DBD527E071E92400652
:10C4F0002E32EC0C2D7E142D12151D8C0F32309E19
:10C500001D8C0A1C049CD3A5001A1D2A221D041789
:10C510001C0794714A076268D64B1D12301C0749EC
:10C52000855A4749C5A44C1E0208472EA1244D43F5
:10C530003103021F29040A054E6134031F734C6046
:10C540002C2ED5F81A11062E15A2052D940A2D8829
:10C55000142D5E1D14092124190308A208814E1E02
:10C5600020160F1F8110385610095AA97BAD83ACD5
:10C57000942DA01C08AB9C6EB531C5B3200316D416
:10C58000402EEE800A2D700F2F94920C033DFE0C6E
:10C590001D8A05253C2DA6121C079CB28C0F732CFE
:10C5A00098571C066841642040A8411C04A96AA948
:10C5B000404B3E85E24B1EE342482C0A2439443965
:10C5C00044312428C2A03725E815442C04605227A2
:10C5D000480B1D18191F93BDE85B2D96163F4A891D
:10C5E0004A0E1D0C171DCE151D0E171F31A64E0429
:10C5F0001C046421235A041D865A1DEE511C04C9D3
:10C60000732AF64D1C0CAC83AB7329A46EBD31CDDF
:10C61000D392311ED420072D28151C04518450AC10
:10C62000031DBC062DEA0431021E91961F353A1CEB
:10C630000B83CE945020A2394428E17A341C048024
:10C640005A27E0332C06276A885A27D2491E416EA2
:10C65000583241AA1D96491DDE5711083D7E041D22
:10C66000A6401C04A29470F0152E3292162FBD9491
:10C67000E0061D741B1E88D00B1DBC0B1C05420858
:10C680004208B2172C06C731C629648E201C074AFF
:10C6900005734A732A84501DD25424086AC85A4527
:10C6A00049C3A4401E937A0C1C04D4A5123C0E1955
:10C6B0006E1D7C0C21A03250A03E7100121D8C0C0E
:10C6C0002D78091C0594504A074A041D5E581DB276
:10C6D000451DFA4C153A1C082351A5498559E68099
:10C6E000342EE6C84D211C1D964E1D704E1D5C411A
:10C6F0002F401810051DAE351D2A0D2E70141E1D5D
:10C70000AA062E9310192DC01C1D982225E63D5413
:10C71000183DF8181FC54AEA4D1DF60D10066A7B34
:10C720004A6AE9A41C082A7B4A62665204F02C1E5D
:10C73000AF70291C0631C5B4AD536E193D0A1A31CC
:10C74000963E514A0B11A815E82D620E2C06AD8CB1
:10C750000F8BEFF83E1D0C031C048120A1F6501F27
:10C760008541E24D2F41233E421DB44B1D8E491E93
:10C770002040352E41225C1004443923081C044417
:10C780003924280315EC2C0B52489C91736CACF2A5
:10C79000BD7460092FDEB8B0531D5E211DB8151D94
:10C7A0003C231D540D1DF6542E685E501C118BCC7D
:10C7B0008BAB836A838B6AE95A476AC973098E4EC9
:10C7C0001E66362E1C048FB5117E0C1DDC0515343B
:10C7D0003E1036092D3809253A3E71D6103D3010ED
:10C7E0001D26272E91A60315C02C086028E23924A7
:10C7F000418596371C08390351E651E5416A501DC1
:10C8000016461C06887B2A7B0A3C442E27004D15C1
:10C81000F23284A22D864B1EA20C0A1E88822F1E85
:10C82000D5660E1C0697CE357B6C42041C0A0A6B3B
:10C830002A62E96B2A6B4AB6111DFA16138BAC9E5D
:10C8400031021F5A6700401C0A607B4B6AA8836A4A
:10C850006AC7FE4D1E8F3A0B1C0410B5522E2F1CBA
:10C8600005308C3084EA1B3D840C2E30DC192D02FF
:10C870001C1DC41A1C08CE8C309C915A89C6502DA0
:10C8800064341D3C5A2C04414439C0351EC2EA3878
:10C890001C064351E572C9E44E180E0D93CC93ACBF
:10C8A0009BED93AC830A72E9941DC64B2D2E0316A3
:10C8B00039F41C0910205207A4D2BD74EA062E36A2
:10C8C000B20F1D30571DAA111383AC981E4E34238E
:10C8D00030044E8C0D9C1DB6111C0562A920A17E52
:10C8E0003611A01D165B1FE9832E302DA2051FAC4B
:10C8F000AFD6251E112256168D402DB4102E0FBC1A
:10C900000F1E5A8A041DC60D11A02DA0121F83CE22
:10C91000C4062C04A210209A491F39241A4A1D9AD1
:10C92000371F5185784C10066BA42E9BED022DB657
:10C930004D1D5A4E1D56491C07AC8B8C8B6B7B8250
:10C94000511D38031DDC032D105B20071840942F68
:10C95000C5B59E1C07AD32A4F172EBE40D1E6CA0B0
:10C9600003240ACC7B8A83EC8BEC8C0C3A1C056A82
:10C97000A828C1BA343220021C040028C1060E2C9B
:10C98000062993EC9C2E42061C05A4AFACF0B20E17
:10C990003F8D7B501C2D5C081D341A1C044D83EF09
:10C9A00042561F6D83640C1F9491A4521E812E0663
:10C9B00015DA19FE1DB2352DB44315302D6E471E04
:10C9C0008B904F1C044DAC4DD24B3D5A4B2D7E4E9F
:10C9D00027832AEC2C0572E96267F6522C0D30E2AF
:10C9E00018405207ACF29C70ACF19C163C0730E347
:10C9F00062897B4CEE1226ED3C2C07732A5A4720A5
:10CA000080F6351DBA3E1D32071D74081C066008ED
:10CA10000049A5440F14056B93ED945E200983AB88
:10CA20005A4662A862CA023DE41D1D20203D020F45
:10CA3000319E1C059CB241C61E0B1D16512D96370A
:10CA40001C052080184000501C07E9834B8B4B9B32
:10CA500092402D2A411D5E3F3C088A8B0872876AEE
:10CA60004598331EA4B64F1E0540521C044762670A
:10CA7000D05014040641A51A2C0420838D76181D6D
:10CA800064192F0D08803B3EA194501004A531027B
:10CA9000962E0092362D4E452D900431A41C0A602E
:10CAA000186010006AC972E90A0E2C0A2A7B6A73A0
:10CAB000297B6B62C8D0561D6C591C06885AEA7BCC
:10CAC000CE280D1DAC12153C1C06109C913145C49E
:10CAD0000B1DE2531C06312431231098381F396492
:10CAE00028522C04C9834BAE481DCA3C1D90471DDB
:10CAF0005446100887726661C45162021C0483495F
:10CB0000225E431DF6321F390152321C04E55A26BB
:10CB10003A591E23DC034E23601520058BED0820B7
:10CB20000225CA1E18EC382D8E362D92363DAA09E4
:10CB30001DF0451D96042A41481DE64B2E8010131A
:10CB40001DD2161C040D83AB4E061C06CD734C6A19
:10CB5000EA74571C062B738D840EA45A1D46122DA1
:10CB600054043329039E3804C32903802C0C6131FB
:10CB70000251E65A4772EA8B6B0C032DDA4B1C0705
:10CB800083099BABAC4E6A4C2C066EBCAFB46F40B5
:10CB9000461F9BED8A411DF8321C074962414249FC
:10CBA000C402581688281C05606AC9831E141F8396
:10CBB000ACCA061DC60A219011881804621021D63D
:10CBC00029DC21A02E61FC4E2D2C0C1DE44B1E8077
:10CBD000E24522A0A01F8BCC0E2F1DDE1A2C05943F
:10CBE000508BEF8817119E1D021925442C044A080A
:10CBF0000864473E82F2072D1E032EA10A54100539
:10CC00005A075A06741D0C5411021E477A471D78A4
:10CC10003D2EA4325031021D7E3D1D024511AA1C3D
:10CC20000AAFB4D0B4D09BED72E974551E47725F61
:10CC30001DE84A2DB81411A01D0464BC04C2D3041D
:10CC400028645E081C640136010235033812AA010B
:04CC50002177000048
:0400000508000131BD
:00000001FF
